:10A668000A594F552041524520464F4F4C20212131
:09A67800212121212121210A00E8
:10A57000420A170001420A290001420A2B00014247
:10A580000A4400004208000000420E1B000042077F
:10A59000D600015607DD00000000000000000000AA
:10A5A000000000000000000000000000560A2E001D
:10A5B000000000000000000000000000000000009B
:10A5C0000000000000410E1A80410A2700410A5293
:10A5D000004107D900440A48010101014807F3007E
:10A5E000351405120303804107FC06C120C124C1B4
:10A5F00022C12BC128C121C12DC123C1ACC1A5C11C
:10A6000029C126C127C12A410E20004107D300419C
:10A6100007FB004102D200410E1F00410A500041D9
:10A6200007FE014107FD014107FF804102D10041C2
:10A630000E2301410A5101410A2D014102CE004180
:10A640000E1D00410A28004102CD004107DA0041F9
:10A6500007DC00410E1E004102CB004107D800413B
:07A6600007DB00410A530073
:100026007F0A1201DD120199120199129EB0C204D3
:10003600C2039007FE7401F0C202E49002D1F0D22E
:1000460005D20C900E1DF0900A27E05407F090F1AF
:10005600FCF012A1C01201599002CCE0640F6003BB
:10006600128DE4128F8E9007F3E0D394604021E462
:10007600F0A37435F0A37414F0A37405F0A37412FE
:10008600F0A37403F0A37401F0A37480F0128DE45E
:10009600125BD17590F0D2AFC288D2A8758921754E
:1000A6008DFD758BFD7598D8758780C2ABD28ED2C3
:1000B600ACD200900A507404F07F0A1201DD3000C1
:1000C60003126F009007FBE0FF6027B40F107F0359
:1000D6001288BF126DAE12015912A214800F90073A
:1000E600FBE0B41F05126EA98003126EBBE49007F5
:1000F600FBF0300403300103300318125E949002C3
:10010600D1E0B4010B1286FA300C0812858A8003FE
:10011600124D46300912125BD1129079A206B392A3
:10012600067F051201DD800C128F8E125BD1122B19
:100136004E12A1C0200287200884200481300B03C0
:100146000200C49007F3E060030200C412A2140286
:0301560000C422C0
:100159001202741203741209B420040330032190AB
:1001690002D1E014600E14600F1460102403701F94
:100179001214C62212245F2212199922121EB322C6
:1001890012220A120FC1122659122C6612001B22C2
:100199009007DBE0701B900E1AE0442090F800F005
:1001A9007F787E00120237900E1AE054DF90F80033
:0201B900F02232
:1001BB009007DBE0701B900E1AE0442090F800F0E3
:1001CB007F1E7E00120237900E1AE054DF90F8006B
:0201DB00F02210
:1001DD00CBEFCBE4900000F0A3F0EBFF7E007C01B1
:1001ED007DF412BBE0900000E0FCA3E0FDC39FECAA
:1001FD009E5036900003E02DF0900002E03CF0A3FD
:10020D00E004F07006900002E004F0900003E004BA
:10021D00F07006900002E004F0900001E004F07030
:0A022D0006900000E004F080B1220A
:10023700758921758CFC758A17D28CE4900004F0BF
:10024700A3F0C3900005E09F900004E09E501B3090
:100257008DFD758CFC758A17C28D900005E004F042
:0D0267007006900004E004F080D8C28C22E4
:100274007F021201DD90F4017440F090F4007435B3
:10028400F07487F0740FF07428F07433F074F0F0A5
:100294007428F0E4F0A37444F090F400E4F0F074F3
:1002A400F0F0E4F07427F074F0F07480F0744DF022
:1002B4007480F0744DF0A3745AF090F400E4F0A349
:1002C400745BF090F400740DF0A3745DF090F4008E
:1002D4007407F07480F0A3745CF090F400E4F0749C
:1002E40050F0A37459F090F4007416F01202F42242
:1002F400E4FFFE1200067F037E0012035090F40117
:100304007442F0754225754380E5431543AE42704F
:100314000215424E600790F400E4F080EC7F007E0A
:10032400271200067F037E0012035090F4017442EA
:10033400F0754225754380E5431543AE42700215BE
:0C034400424E600790F400E4F080EC22D0
:0E00060090F4017446F0EF90F400F0EEF0225A
:10035000EE701CEF14600E14600F14601024037014
:100360000E744E800A744F8006744D8002744C9057
:04037000F401F02282
:0700140090F4017442F02298
:1003740075420275430A754454E4900006F0A3F0F4
:10038400900006E0FEA3E0FFC39428EE9400501D05
:1003940074542FF582EE340AF58374FFF09000074D
:1003A400E004F07006900006E004F080D37FD07E75
:1003B400297D037C007B287A0012096E9002D1E02B
:1003C40064016073E4900006F0A3F0900006E0FE80
:1003D400A3E0FFC394B3EE9400501D74542FF58230
:1003E400EE340AF583740CF0900007E004F0700614
:1003F400900006E004F080D320040330032A900226
:10040400D1E0640260117F0B7E2A7D017C007BB306
:100414007A0012096E80207F0B7E2A7D017C007B8E
:100424008D7A0012096E800F7F057E2A7D017C0083
:100434007BB37A0012096EE4900006F0A3F09000FA
:1004440006E0FEA3E0FFC39428EE9400501D74540C
:100454002FF582EE340AF58374FFF0900007E00470
:10046400F07006900006E004F080D37FC87E457DDE
:10047400037C007B287A0012096EE4900006F0A346
:10048400F0900006E0FEA3E0FFC39478EE940050E1
:100494001D74542FF582EE340AF58374FFF0900036
:1004A40007E004F07006900006E004F080D37FC0FB
:1004B4007E487D037C007B787A0012096EE490000C
:1004C40006F0A3F0900006E0FEA3E0FFC39412EE52
:1004D4009400501D74542FF582EE340AF583740190
:1004E400F0900007E004F07006900006E004F0804D
:1004F400D37FF97E457D017C007B127A0012096E60
:100504003004030205B99002D1E0640170030205CE
:10051400B93003030205B9E4900006F0A3F090009B
:1005240006E0FEA3E0FFC3940DEE9400501D745446
:100534002FF582EE340AF58374FFF0900007E0048F
:10054400F07006900006E004F080D374542FF58216
:10055400EE340AF58374FCF07F407E2D7D037C002D
:100564007B0E7A0012096E7F907E2D7D037C007BCA
:100574000E7A0012096E200B3C7F277E2D7D037CB2
:10058400007B077A0012096E7F777E2D7D037C0045
:100594007B077A0012096E7F9F7E2D7D037C007B92
:1005A400077A0012096E7FC77E2D7D037C007B07CE
:1005B4007A0012096E9002D1E064016003020856C9
:1005C40075420275430A754454900006F0A3F0C3C3
:1005D400900007E0943C900006E094005023AB4266
:1005E4000544E544AA437002054314F9740112BB9F
:1005F400CC900007E004F07006900006E004F08060
:10060400CEAB420544E544AA437002054314F97491
:100614000F12BBCCE4900006F0A3F0C3900007E0F7
:100624009406900006E094005023AB420544E54450
:10063400AA437002054314F9740112BBCC9000075D
:10064400E004F07006900006E004F080CEAB4205B2
:1006540044E544AA437002054314F9740F12BBCC59
:10066400AB420544E544AA437002054314F97407F8
:1006740012BBCCAB420544E544AA437002054314C3
:10068400F9740312BBCCAB420544E544AA4370029F
:10069400054314F9740112BBCC7F537E40E4FDFC86
:1006A4007B47FA12096E900A5474F0F0A374E0F0D8
:1006B400A374C0F0A37480F07FDC7E35E4FDFC7B82
:1006C40004FA12096EE4900006F0A3F0900006E02C
:1006D400FEA3E0FFC39421EE9400501D74542FF543
:1006E40082EE340AF58374FFF0900007E004F070A2
:1006F40006900006E004F080D37F547E407D037CA6
:10070400007B217A0012096E900A547480F0A3745D
:10071400C0F0A374E0F0A374F0F0A3F0A374E0F0CD
:10072400A374C0F0A37480F07FD57E3F7D017C006C
:100734007B087A0012096EE4900006F0A3F09000A2
:1007440006E0FEA3E0FFC39404EE9400501D74542D
:060754002FF582EE340ACD
:10075A00F5837401F0900007E004F070069000063B
:10076A00E004F080D37F9B7E407D017C007B047A8D
:10077A000012096EE4900006F0A3F0900006E0FE75
:10078A00A3E0FFC3941FEE9400501D74542FF5820A
:10079A00EE340AF58374FFF0900007E004F0700667
:1007AA00900006E004F080D37F9D7E2A7D037C00C2
:1007BA007B1F7A0012096E7F257E347D037C007BC5
:1007CA001F7A0012096EE4900006F0A3F09000066A
:1007DA00E0FEA3E0FFC3943CEE9400501D74542F36
:1007EA00F582EE340AF5837480F0900007E004F095
:1007FA007006900006E004F080D37FC57E2A7D0152
:10080A007C007B3C7A0012096EE4900006F0A3F0AB
:10081A00900006E0FEA3E0FFC3943CEE9400501D56
:10082A0074542FF582EE340AF5837401F0900007B0
:10083A00E004F07006900006E004F080D37FE37EC7
:10084A002A7D017C007B3C7A0012096EE490000A42
:10085A00F0A3F0C390000BE0940490000AE0940027
:10086A004003020906E4900008F0A3F0C3900009CF
:10087A00E09408900008E094005070E4900006F0BC
:10088A00A3F0900006E0FEA3E0FFC39412EE9400EA
:10089A00501D74542FF582EE340AF58374FFF090DC
:1008AA000007E004F07006900006E004F080D390A0
:1008BA00000AE0FEA3E0FF7C007D0A12BBE0EF2401
:1008CA0089FFEE3449FE900009E02FFF900008E00E
:1008DA003EFE7D017B127A0012096E900009E00447
:1008EA00F07006900008E004F0808190000BE004AC
:0D08FA00F0700690000AE004F002085D2294
:100907008F429007D6E07004A3E06401705890000E
:100917000CF090000CE0FFC39412501474542FF5A0
:1009270082E4340AF583E4F090000CE004F080E2FE
:10093700E490000DF090000DE0FDC394085027E50A
:100947004275F00AA42489FFE5F03449FE7C00EFE4
:100957002DFFEC3EFE7D017B127A0012096E90009E
:070967000DE004F080CF2237
:10096E008C458D46120006AF46AE4512035012005E
:10097E0014E490000EF0A3F090000EE0FEA3E0FF52
:10098E00C39BEE9A501F74542FF582EE340AF583F2
:10099E00E090F400F090000FE004F0700690000E6E
:0609AE00E004F080D322FA
:1009B400900A48E014605A147003020A5714700332
:1009C400020A9824036003020AD7E4FF120907907D
:1009D40002D3E4F0A37420F0A3E4F0A37420F0A302
:1009E400E4F0A37420F0A3E4F0A37420F0A3E4F0F3
:1009F400A37420F0A3E4F0A37420F0A3E4F0A374A0
:100A040020F0A3E4F0A37420F0E4A3F0A3F0020A1E
:100A1400D79002D3E4F0A37420F0A3E4F0A37420ED
:100A2400F0A3E4F0A37454F0A3E4F0A37465F0A37A
:100A3400E4F0A37473F0A3E4F0A37474F0A3E4F0FB
:100A4400A37420F0A3E4F0A37420F0E4A3F0A3F0D3
:100A5400020AD79002D3E4F0A37420F0A3E4F0A335
:100A64007452F0A3E4F0A37465F0A3E4F0A37474E7
:100A7400F0A3E4F0A37475F0A3E4F0A37472F0A3FC
:100A8400E4F0A3746EF0A3E4F0A37420F0E4A3F004
:100A9400A3F0803F9002D3E4F0A37420F0A3E4F029
:100AA400A37420F0A3E4F0A37420F0A3E4F0A374EF
:100AB4004EF0A3E4F0A3746FF0A3E4F0A37420F069
:100AC400A3E4F0A37420F0A3E4F0A37420F0E4A35F
:100AD400F0A3F07FB17E221210D8900A49E014608E
:100AE4005A147003020B81147003020BC2240360B6
:100AF40003020C017F011209079002D3E4F0A374EE
:100B040020F0A3E4F0A37420F0A3E4F0A37420F095
:100B1400A3E4F0A37420F0A3E4F0A37420F0A3E40E
:100B2400F0A37420F0A3E4F0A37420F0A3E4F0A3F2
:100B34007420F0E4A3F0A3F0020C019002D3E4F0DB
:100B4400A37420F0A3E4F0A37453F0A3E4F0A3741B
:100B540065F0A3E4F0A37474F0A3E4F0A37475F057
:100B6400A3E4F0A37470F0A3E4F0A37420F0A3E46E
:100B7400F0A37420F0E4A3F0A3F0020C019002D3DC
:100B8400E4F0A37420F0A3E4F0A37444F0A3E4F02D
:100B9400A37465F0A3E4F0A3746CF0A3E4F0A3746D
:100BA40065F0A3E4F0A37474F0A3E4F0A37465F017
:100BB400A3E4F0A37420F0E4A3F0A3F0803F900238
:100BC400D3E4F0A37420F0A3E4F0A37453F0A3E4FB
:100BD400F0A37474F0A3E4F0A3746FF0A3E4F0A39F
:100BE4007472F0A3E4F0A37465F0A3E4F0A374209A
:100BF400F0A3E4F0A37420F0E4A3F0A3F07FBB7EA1
:100C0400221210D8900A4AE0146066147003020C91
:100C1400B7147003020CF9147003020D3B14700333
:100C2400020D7C24056003020DBB7F0212090790AC
:100C340002D3E4F0A37420F0A3E4F0A37420F0A39F
:100C4400E4F0A37420F0A3E4F0A37420F0A3E4F090
:100C5400A37420F0A3E4F0A37420F0A3E4F0A3743D
:100C640020F0A3E4F0A37420F0E4A3F0A3F0020DB9
:100C7400BB9002D3E4F0A37420F0A3E4F0A3745275
:100C8400F0A3E4F0A37465F0A3E4F0A37463F0A309
:100C9400E4F0A3746FF0A3E4F0A37472F0A3E4F09F
:100CA400A37464F0A3E4F0A37420F0E4A3F0A3F02D
:100CB400020DBB9002D3E4F0A37420F0A3E4F0A3EC
:100CC4007443F0A3E4F0A3746CF0A3E4F0A374659C
:100CD400F0A3E4F0A37461F0A3E4F0A37472F0A3AE
:100CE400E4F0A37420F0A3E4F0A37420F0E4A3F0F0
:100CF400A3F0020DBB9002D3E4F0A37450F0A3E47C
:100D0400F0A37472F0A3E4F0A37465F0A3E4F0A379
:100D14007476F0A3E4F0A37469F0A3E4F0A3746F11
:100D2400F0A3E4F0A37475F0A3E4F0A37473F0E407
:100D3400A3F0A3F0020DBB9002D3E4F0A37449F036
:100D4400A3E4F0A3746EF0A3E4F0A37463F0A3E44B
:100D5400F0A37472F0A3E4F0A37465F0A3E4F0A329
:100D64007461F0A3E4F0A37473F0A3E4F0A37465D6
:100D7400F0E4A3F0A3F0803F9002D3E4F0A3745214
:100D8400F0A3E4F0A37465F0A3E4F0A3742DF0A33E
:060D9400E4F0A37474F00A
:100D9A00A3E4F0A37472F0A3E4F0A37461F0A3E4F3
:100DAA00F0A37469F0A3E4F0A3746EF0E4A3F0A3D3
:100DBA00F07FC57E221210D8900A4BE0B40700409B
:100DCA0003020FB9900DD5F8282873020DEA020E16
:100DDA0031020E73020EB5020EF7020F39020F7AB4
:100DEA007F031209079002D3E4F0A37420F0A3E46E
:100DFA00F0A37420F0A3E4F0A37420F0A3E4F0A31A
:100E0A007420F0A3E4F0A37420F0A3E4F0A3742008
:100E1A00F0A3E4F0A37420F0A3E4F0A37420F0E4B8
:100E2A00A3F0A3F0020FB99002D3E4F0A37453F035
:100E3A00A3E4F0A37465F0A3E4F0A3746CF0A3E454
:100E4A00F0A37466F0A3E4F0A37454F0A3E4F0A34F
:100E5A007465F0A3E4F0A37473F0A3E4F0A37474CC
:100E6A00F0E4A3F0A3F0020FB99002D3E4F0A37464
:100E7A0020F0A3E4F0A37420F0A3E4F0A37456F0E6
:100E8A00A3E4F0A37469F0A3E4F0A37465F0A3E407
:100E9A00F0A37477F0A3E4F0A37420F0A3E4F0A322
:100EAA007420F0E4A3F0A3F0020FB99002D3E4F0A7
:100EBA00A37420F0A3E4F0A37420F0A3E4F0A374D5
:100ECA004EF0A3E4F0A37465F0A3E4F0A37478F001
:100EDA00A3E4F0A37474F0A3E4F0A37420F0A3E4F1
:100EEA00F0A37420F0E4A3F0A3F0020FB99002D3A8
:100EFA00E4F0A37420F0A3E4F0A37420F0A3E4F0D8
:100F0A00A37459F0A3E4F0A37465F0A3E4F0A37406
:100F1A0073F0A3E4F0A37420F0A3E4F0A37420F028
:100F2A00A3E4F0A37420F0E4A3F0A3F0020FB990B5
:100F3A0002D3E4F0A37444F0A3E4F0A37465F0A32D
:100F4A00E4F0A37463F0A3E4F0A37472F0A3E4F0F2
:100F5A00A37465F0A3E4F0A37461F0A3E4F0A374AE
:100F6A0073F0A3E4F0A37465F0E4A3F0A3F0803F68
:100F7A009002D3E4F0A37420F0A3E4F0A37443F046
:100F8A00A3E4F0A3746CF0A3E4F0A3746FF0A3E4F9
:100F9A00F0A37473F0A3E4F0A37465F0A3E4F0A3E0
:100FAA007420F0A3E4F0A37420F0E4A3F0A3F07F8C
:070FBA00CF7E221210D822A5
:100FC100E4900010F0900010E0FFC39414501474EA
:100FD100542FF582E4340AF583E4F0900010E00424
:100FE100F080E2E4900011F0900011E0FFC3940A58
:100FF1005045EF24FAFFE4342EFE7D017C007B1482
:101001007A0012096E900011E024E2FFE43432FE0E
:1010110012096E900011E024CAFFE43436FE120971
:101021006E900011E024B2FFE4343AFE12096E9092
:101031000011E004F080B1E4900010F0900010E0A5
:10104100FFC39414501574542FF582E4340AF583C8
:1010510074FFF0900010E004F080E1E4900011F0E2
:10106100900011E0F9C3940A506C9007FEE024FE51
:10107100601F14603114604324037052E924FAFFA5
:10108100E4342EFE7D017C007B147A0012096E800F
:101091003DE924E2FFE43432FE7D017C007B147AD9
:1010A1000012096E8028E924CAFFE43436FE7D016E
:1010B1007C007B147A0012096E8013E924B2FFE4EC
:1010C100343AFE7D017C007B147A0012096E900097
:0710D10011E004F0808A2207
:1010D8008E458F46E4900018F0A3F0A3F0A3F075B6
:1010E800470275480A754954900019E025E0FF90B9
:1010F8000018E033FE74D32FF582EE3402F583E056
:10110800FEA3E04E6010900019E004F07006900015
:1011180018E004F080D2E4900016F0A3F0900014D8
:10112800F0A3F0900018E0FEA3E0FF900014E0FCAC
:10113800A3E0FDC39FEC9E400302127EED25E0FF75
:10114800EC33FE74D32FF582EE3402F583E0FEA370
:10115800E0D3947EEE940040030211F0E490001274
:10116800F0A3F0900012E0FCA3E0FDC39410EC940F
:10117800005064900015E025E0FF900014E033FE75
:1011880074D32FF582EE3402F583A3E0C4F8540F2C
:10119800C868FF0582D5820215831582E0C454F021
:1011A80048FEED2FFFEC3EFE74812FF582EE34A64B
:1011B800F583E493FFAB470549E549AA4870020562
:1011C8004814F9EF12BBCC900013E004F0700690BD
:1011D8000012E004F0808C900017E004F070069094
:1011E8000016E004F002126DE4900012F0A3F090F3
:1011F8000012E0FCA3E0FDC39420EC94005058904A
:101208000015E025E0FF900014E033FE74D32FF5BD
:1012180082EE3402F583E0FEA3E07805C333CE33D3
:10122800CED8F92DFFEC3EFE74912FF582EE349E58
:10123800F583E493FFAB470549E549AA48700205E1
:101248004814F9EF12BBCC900013E004F07006903C
:101258000012E004F08098900017E02402F090005B
:1012680016E03400F0900015E004F07006900014C9
:10127800E004F002112B75470275480A754954E4D9
:10128800900018F0A3F0900016E0FEA3E0FFC390D2
:101298000019E09F900018E09E507890001BE02510
:1012A80046FF90001AE03545FE1200067F017E00D9
:1012B80012035090F4017442F0E4900012F0A3F08D
:1012C800C3900013E09410900012E094005025ABF6
:1012D800470549E549AA487002054814F912BBB107
:1012E80090F400F0900013E004F07006900012E013
:1012F80004F080CC90001BE004F0700690001AE027
:1013080004F0900019E004F07006900018E004F072
:0A13180002128EAB47AA48A9492231
:101322008E368F37E4900022F0A3F0A3F0A3F0757D
:10133200380275390A753A54900022F0A3F09000F1
:1013420023E025E0FF900022E033FE74D32FF582E4
:10135200EE3402F583E0FEA3E04E6010900023E03D
:1013620004F07006900022E004F080D2E4900020A5
:10137200F0A3F090001EF0A3F0900022E0FEA3E0A4
:10138200FFC390001FE09F90001EE09E40030214E6
:1013920028E490001CF0A3F090001CE0FCA3E0FD08
:1013A200C39448EC9400505F90001FE025E0FF904A
:1013B200001EE033FE74D32FF582EE3402F583E093
:1013C200FEA3E0F5828E83744812BEA4E5822DF559
:1013D20082EC3583F583E5822471F582E58334AEB0
:1013E200F583E493FFAB38053AE53AAA3970020572
:1013F2003914F9EF12BBCC90001DE004F070069096
:10140200001CE004F08091900021E02403F09000A1
:1014120020E03400F090001FE004F0700690001EFF
:10142200E004F002137B75380275390A753A54E408
:10143200900022F0A3F0900020E0FEA3E0FFC39012
:101442000023E09F900022E09E5078900025E02546
:1014520037FF900024E03536FE1200067F017E0041
:1014620012035090F4017442F0E490001CF0A3F0D7
:10147200C390001DE0941890001CE094005025AB2E
:1014820038053AE53AAA397002053914F912BBB1A6
:1014920090F400F090001DE004F0700690001CE053
:1014A20004F080CC900025E004F07006900024E067
:1014B20004F0900023E004F07006900022E004F0B3
:0414C20002143822B6
:1014C6009002D3E4F0A37453F0A3E4F0A37474F091
:1014D600A3E4F0A37461F0A3E4F0A37474F0A3E4AE
:1014E600F0A37475F0A3E4F0A37473F0A3E4F0A37F
:1014F600743AF0E4A3F0A3F0FFFE1210D89002D3E2
:10150600E4F0A3745BF0A3E4F0A37420F0A3E4F08A
:10151600A37444F0A3E4F0A3746FF0A3E4F0A374FF
:1015260077F0A3E4F0A3746EF0A3E4F0A37453F091
:10153600A3E4F0A37474F0A3E4F0A37472F0A3E43C
:10154600F0A37465F0A3E4F0A37461F0A3E4F0A340
:10155600746DF0A3E4F0A37420F0A3E4F0A3745D2B
:10156600F0E4A3F0A3F07FC37E031210D89002D359
:10157600E4F0A37420F0A3E4F0A3745BF0A3E4F01A
:10158600A37420F0A3E4F0A37455F0A3E4F0A374CD
:1015960070F0A3E4F0A37453F0A3E4F0A37474F022
:1015A600A3E4F0A37472F0A3E4F0A37465F0A3E4DB
:1015B600F0A37461F0A3E4F0A3746DF0A3E4F0A3C8
:1015C6007420F0A3E4F0A3745DF0E4A3F0A3F07F2D
:1015D600D77E031210D89002D3E4F0A37446F0A38A
:1015E600E4F0A37441F0A3E4F0A37453F0A3E4F091
:1015F600A37454F0A3E4F0A3743AF0E4A3F0A3F0C8
:101606007F307E071210D87F447E071210D89002D2
:10161600D3E4F0A3746BF0A3E4F0A37462F0A3E444
:10162600F0A37470F0A3E4F0A37473F0E4A3F0A342
:10163600F07F3F7E071210D87F537E071210D89096
:1016460002D3E4F0A37449F0A3E4F0A3744EF0A32C
:10165600E4F0A37454F0A3E4F0A37452F0A3E4F00E
:10166600A3744CF0A3E4F0A37456F0A3E4F0A374BF
:1016760044F0A3E4F0A3743AF0E4A3F0A3F07F509F
:101686007E0A1210D87F647E0A1210D89002D3E424
:10169600F0A3746BF0A3E4F0A37462F0A3E4F0A3E8
:1016A6007470F0A3E4F0A37473F0E4A3F0A3F07FE6
:1016B6005F7E0A1210D87F737E0A1210D89002D36A
:1016C600E4F0A3744DF0A3E4F0A37441F0A3E4F0B6
:1016D600A37458F0A3E4F0A37452F0A3E4F0A37447
:1016E60041F0A3E4F0A37454F0A3E4F0A37445F02E
:1016F600A3E4F0A3743AF0E4A3F0A3F07F707E0DA8
:101706001210D87F847E0D1210D89002D3E4F0A375
:10171600746BF0A3E4F0A37462F0A3E4F0A3747016
:10172600F0A3E4F0A37473F0E4A3F0A3F07F7F7E4C
:101736000D1210D87F937E0D1210D89002D3E4F0CC
:10174600A3744DF0A3E4F0A37441F0A3E4F0A374F2
:1017560052F0A3E4F0A37447F0A3E4F0A37449F0B5
:10176600A3E4F0A3744EF0A3E4F0A3743AF0E4A368
:10177600F0A3F07F907E101210D87FA47E10121076
:10178600D89002D3E4F0A37464F0A3E4F0A3744207
:10179600F0A3E4F0A37420F0E4A3F0A3F07FA07E0E
:1017A600101210D87FB47E101210D89002D3E4F035
:1017B600A37450F0A3E4F0A3744FF0A3E4F0A37471
:1017C60057F0A3E4F0A37445F0A3E4F0A37452F039
:1017D600A3E4F0A3743AF0E4A3F0A3F07FB07E1381
:1017E6001210D87FC47E131210D89002D3E4F0A34F
:1017F6007464F0A3E4F0A37442F0A3E4F0A3746D60
:10180600F0E4A3F0A3F07FC07E131210D87FD47E3D
:10181600131210D89002D3E4F0A37441F0A3E4F0BD
:10182600A37454F0A3E4F0A37454F0A3E4F0A374F7
:1018360045F0A3E4F0A3744EF0A3E4F0A3743AF0E9
:10184600E4A3F0A3F07FD07E161210D87FE47E16B4
:101856001210D89002D3E4F0A37464F0A3E4F0A3CA
:101866007442F0A3E4F0A37420F0E4A3F0A3F07FA5
:10187600E07E161210D87FF47E161210D89002D38E
:10188600E4F0A37443F0A3E4F0A37441F0A3E4F0FE
:10189600A37450F0A3E4F0A37441F0A3E4F0A3749E
:0618A60043F0A3E4F0A3EF
:1018AC007449F0A3E4F0A37454F0A3E4F0A37459C6
:1018BC00F0A3E4F0A3743AF0E4A3F0A3F07FF07E7D
:1018CC00191210D87F047E1A1210D89002D3E4F0AB
:1018DC00A37425F0E4A3F0A3F07F017E1A1210D8B4
:0B18EC007F157E1A1210D81218F72288
:1018F700E4FFEFC3941D501875F002EFA424D3F54D
:1019070082E5F03402F583E4F0A37420F00F80E25F
:101917009002DDE4F0A3743AF09002D7E4F0A374E8
:101927003AF09002EFE4F0A3742FF09002E9E4F0AC
:10193700A3742FF09002F1E4F0A37432F0A3E4F063
:10194700A37430F0E490030DF0A3F07F237E1F1201
:1019570010D89002D3E4F0A3743CF0A3E4F0A3748E
:1019670041F0A3E4F0A37454F0A3E4F0A37455F09A
:10197700A3E4F0A3745FF0A3E4F0A37452F0A3E42C
:10198700F0A3743EF0E4A3F0A3F07F197E1F1210BA
:02199700D82254
:10199900E4900026F09002D3F0A37453F0A3E4F08E
:1019A900A37474F0A3E4F0A37461F0A3E4F0A37446
:1019B90074F0A3E4F0A37475F0A3E4F0A37473F0D6
:1019C900A3E4F0A3743AF0E4A3F0A3F0FFFE12102D
:1019D900D89002D3E4F0A3745BF0A3E4F0A37420DD
:1019E900F0A3E4F0A37446F0A3E4F0A37461F0A3B8
:1019F900E4F0A37472F0A3E4F0A37420F0A3E4F07C
:101A0900A37445F0A3E4F0A3746EF0A3E4F0A37407
:101A190064F0A3E4F0A37420F0A3E4F0A3745DF0F0
:101A2900E4A3F0A3F07F4B7E031210D89002D3E415
:101A3900F0A3745BF0A3E4F0A37420F0A3E4F0A393
:101A4900744EF0A3E4F0A37465F0A3E4F0A3746109
:101A5900F0A3E4F0A37472F0A3E4F0A37420F0A35C
:101A6900E4F0A37445F0A3E4F0A3746EF0A3E4F0EA
:101A7900A37464F0A3E4F0A37420F0A3E4F0A374C6
:101A89005DF0E4A3F0A3F07F5F7E031210D890020B
:101A9900D3E4F0A37446F0A3E4F0A37445F0A3E4FF
:101AA900F0A37443F0A3E4F0A37420F0A3E4F0A33B
:101AB9007446F0A3E4F0A37441F0A3E4F0A37453D3
:101AC900F0A3E4F0A37454F0A3E4F0A3743AF0E4AF
:101AD900A3F0A3F07F407E061210D87F547E061231
:101AE90010D89002D3E4F0A37446F0A3E4F0A374F1
:101AF90045F0A3E4F0A37443F0A3E4F0A37420F049
:101B0900A3E4F0A37449F0A3E4F0A3744EF0A3E4B2
:101B1900F0A37454F0A3E4F0A37452F0A3E4F0A387
:101B2900743AF0E4A3F0A3F07F607E091210D87F25
:101B3900747E091210D89002D3E4F0A37443F0A381
:101B4900E4F0A37452F0A3E4F0A37443F0A3E4F027
:101B5900A37420F0A3E4F0A37446F0A3E4F0A37403
:101B690041F0A3E4F0A37453F0A3E4F0A37454F098
:101B7900A3E4F0A3743AF0E4A3F0A3F07F807E0C11
:101B89001210D87F947E0C1210D89002D3E4F0A3DF
:101B99007443F0A3E4F0A37452F0A3E4F0A37443F4
:101BA900F0A3E4F0A37420F0A3E4F0A37449F0A334
:101BB900E4F0A3744EF0A3E4F0A37454F0A3E4F0AA
:101BC900A37452F0A3E4F0A3743AF0E4A3F0A3F0F1
:101BD9007FA07E0F1210D87FB47E0F1210D890020A
:101BE900D3E4F0A37448F0A3E4F0A37445F0A3E4AC
:101BF900F0A37443F0A3E4F0A37420F0A3E4F0A3EA
:101C09007446F0A3E4F0A37441F0A3E4F0A3745381
:101C1900F0A3E4F0A37454F0A3E4F0A3743AF0E45D
:101C2900A3F0A3F07FC07E121210D87FD47E1212C7
:101C390010D89002D3E4F0A37448F0A3E4F0A3749D
:101C490045F0A3E4F0A37443F0A3E4F0A37420F0F7
:101C5900A3E4F0A37449F0A3E4F0A3744EF0A3E461
:101C6900F0A37454F0A3E4F0A37452F0A3E4F0A336
:101C7900743AF0E4A3F0A3F07FE07E151210D87F48
:101C8900F47E151210D8E4900026F0900026E0FFAB
:101C9900C39428501574542FF582E4340AF58374DB
:101CA900FFF0900026E004F080E17F007E407D0394
:101CB9007C007B287A0012096E200303021DC8905C
:101CC90002D3E4F0A37453F0A3E4F0A37474F0A373
:101CD900E4F0A3746FF0A3E4F0A37470F0A3E4F04C
:101CE900A37420F0A3E4F0A37474F0A3E4F0A37444
:101CF90069F0A3E4F0A3746DF0A3E4F0A37465F0B4
:101D0900A3E4F0A3743AF0A3E4F0A37420F0A3E4ED
:101D1900F0A37420F0A3E4F0A37420F0A3E4F0A3EB
:101D29007420F0A3E4F0A3742FF0A3E4F0A37420CB
:101D3900F0A3E4F0A37420F0A3E4F0A3742FF0A3BC
:101D4900E4F0A37432F0A3E4F0A37430F0A3E4F058
:101D5900A37420F0A3E4F0A37420F0A3E4F0A37427
:101D690020F0A3E4F0A37420F0A3E4F0A37420F01E
:061D7900A3E4F0A3743A9C
:101D7F00F0A3E4F0A37420F0A3E4F0A37420F0A385
:101D8F00E4F0A3743AF0A3E4F0A37420F0A3E4F01A
:101D9F00A37420F0E4A3F0A3F0900026E0FF7E00F0
:101DAF007C027D8012BBE0EF2435FFEE3403FE1280
:101DBF0010D87FA07E191210D89002D3E4F0A3742C
:101DCF0053F0A3E4F0A37474F0A3E4F0A37461F0F0
:101DDF00A3E4F0A37472F0A3E4F0A37474F0A3E48B
:101DEF00F0A37420F0A3E4F0A37474F0A3E4F0A3C1
:101DFF007469F0A3E4F0A3746DF0A3E4F0A3746529
:101E0F00F0A3E4F0A3743AF0A3E4F0A37420F0A3DA
:101E1F00E4F0A37420F0A3E4F0A37420F0A3E4F0A3
:101E2F00A3742FF0A3E4F0A37420F0A3E4F0A37441
:101E3F0020F0A3E4F0A3742FF0A3E4F0A37432F026
:101E4F00A3E4F0A37430F0A3E4F0A37420F0A3E4B0
:101E5F00F0A37420F0A3E4F0A37420F0A3E4F0A3A4
:101E6F007420F0A3E4F0A37420F0A3E4F0A3743A79
:101E7F00F0A3E4F0A37420F0A3E4F0A37420F0A384
:101E8F00E4F0A3743AF0A3E4F0A37420F0A3E4F019
:101E9F00A37420F0E4A3F0A3F07F207E1C1210D8CF
:041EAF001218F722EC
:101EB3009002D3E4F0A37453F0A3E4F0A37474F09A
:101EC300A3E4F0A37461F0A3E4F0A37474F0A3E4B7
:101ED300F0A37475F0A3E4F0A37473F0A3E4F0A388
:101EE300743AF0E4A3F0A3F0FFFE1210D89002D3EB
:101EF300E4F0A3745BF0A3E4F0A37420F0A3E4F094
:101F0300A37446F0A3E4F0A37461F0A3E4F0A37414
:101F130072F0A3E4F0A37420F0A3E4F0A37445F0FB
:101F2300A3E4F0A3746EF0A3E4F0A37464F0A3E459
:101F3300F0A37420F0A3E4F0A3745DF0E4A3F0A392
:101F4300F07FEC7E031210D89002D3E4F0A3745B0D
:101F5300F0A3E4F0A37420F0A3E4F0A3744EF0A381
:101F6300E4F0A37465F0A3E4F0A37461F0A3E4F0D8
:101F7300A37472F0A3E4F0A37420F0A3E4F0A374B9
:101F830045F0A3E4F0A3746EF0A3E4F0A37464F04B
:101F9300A3E4F0A37420F0A3E4F0A3745DF0E4A33E
:101FA300F0A3F0FF7E041210D89002D3E4F0A374E0
:101FB3004CF0A3E4F0A3744FF0A3E4F0A37453F044
:101FC300E4A3F0A3F07FD77E071210D87FEB7E0740
:101FD3001210D89002D3E4F0A3744CF0A3E4F0A35E
:101FE300744FF0A3E4F0A37446F0E4A3F0A3F07FEE
:101FF300F77E0A1210D8740BFFFE1210D89002D38A
:10200300E4F0A3744CF0A3E4F0A3744FF0A3E4F062
:10201300A37450F0E4A3F0A3F07F177E0E1210D840
:102023007F2B7E0E1210D89002D3E4F0A3744CF0F1
:10203300A3E4F0A37443F0A3E4F0A37444F0A3E493
:10204300F0A37428F0A3E4F0A37446F0A3E4F0A390
:102053007441F0A3E4F0A37453F0A3E4F0A3745425
:10206300F0A3E4F0A37429F0E4A3F0A3F07F377E98
:10207300111210D87F4B7E111210D89002D3E4F0C6
:10208300A3744CF0A3E4F0A37443F0A3E4F0A374AB
:1020930044F0A3E4F0A37428F0A3E4F0A37449F09C
:1020A300A3E4F0A3744EF0A3E4F0A37454F0A3E408
:1020B300F0A37452F0A3E4F0A37429F0E4A3F0A313
:1020C300F07F577E141210D87F6B7E141210D890B5
:1020D30002D3E4F0A3744CF0A3E4F0A3744FF0A391
:1020E300E4F0A3744DF0E4A3F0A3F07F777E17121E
:1020F30010D87F8B7E171210D89002D3E4F0A3740C
:102103001CF0A3E4F0A3741DF0A3E4F0A37420F087
:10211300A3E4F0A37448F0A3E4F0A37469F0A3E488
:10212300F0A37473F0A3E4F0A37474F0A3E4F0A336
:10213300746FF0A3E4F0A37472F0A3E4F0A37479D2
:10214300F0A3E4F0A37420F0A3E4F0A37464F0A379
:10215300E4F0A37465F0A3E4F0A37466F0A3E4F0E1
:10216300A37465F0A3E4F0A37463F0A3E4F0A37491
:1021730074F0E4A3F0A3F07FF97E1B1210D8900251
:10218300D3E4F0A3740CF0A3E4F0A3740DF0A3E480
:10219300F0A37420F0A3E4F0A37443F0A3E4F0A34A
:1021A3007475F0A3E4F0A37472F0A3E4F0A3747263
:1021B300F0A3E4F0A37465F0A3E4F0A3746EF0A3BA
:1021C300E4F0A37474F0A3E4F0A37420F0A3E4F0A8
:1021D300A37464F0A3E4F0A37465F0A3E4F0A37420
:1021E30066F0A3E4F0A37465F0A3E4F0A37463F0D2
:1021F300A3E4F0A37474F0E4A3F0A3F07F0D7E1CBA
:072203001210D81218F72297
:10220A009002D3E4F0A37453F0A3E4F0A37474F03F
:10221A00A3E4F0A37461F0A3E4F0A37474F0A3E45C
:10222A00F0A37475F0A3E4F0A37473F0A3E4F0A32D
:10223A00743AF0A3E4F0A3745CF0A3E4F0A3745C32
:10224A00F0A3E4F0A3744DF0A3E4F0A37465F0A343
:10225A00E4F0A3746EF0A3E4F0A37475F0A3E4F0C1
:10226A00A3745CF0A3E4F0A37454F0A3E4F0A374A1
:10227A0065F0A3E4F0A37473F0A3E4F0A37474F01C
:10228A00A3E4F0A3743FF0A3E4F0A37420F0A3E462
:10229A00F0A37420F0A3E4F0A37420F0A3E4F0A365
:1022AA007420F0A3E4F0A37420F0A3E4F0A3743C38
:1022BA00F0A3E4F0A3744FF0A3E4F0A3744BF0A3EB
:1022CA00E4F0A3743EF0A3E4F0A37420F0A3E4F0D6
:1022DA00A37420F0A3E4F0A37420F0A3E4F0A374A1
:1022EA0020F0A3E4F0A37420F0E4A3F0A3F0FFFE2F
:1022FA001210D89002D3E4F0A37420F0A3E4F0A360
:10230A007420F0A3E4F0A37420F0A3E4F0A3744DC6
:10231A00F0A3E4F0A37445F0A3E4F0A3744EF0A391
:10232A00E4F0A37455F0A3E4F0A37420F0E4A3F05E
:10233A00A3F07F9A7E031210D89002D3E4F0A3741C
:10234A0031F0A3E4F0A3742EF0A3E4F0A37454F0E4
:10235A00A3E4F0A37465F0A3E4F0A37473F0A3E418
:10236A00F0A37474F0A3E4F0A37420F0E4A3F0A340
:10237A00F07F4A7E081210D89002D3E4F0A3743298
:10238A00F0A3E4F0A3742EF0A3E4F0A37453F0A333
:10239A00E4F0A37465F0A3E4F0A37474F0A3E4F08A
:1023AA00A37475F0A3E4F0A37470F0E4A3F0A3F0AF
:1023BA007F327E0C1210D89002D3E4F0A37433F06B
:1023CA00A3E4F0A3742EF0A3E4F0A37452F0A3E400
:1023DA00F0A37465F0A3E4F0A37463F0A3E4F0A39C
:1023EA00746FF0A3E4F0A37472F0A3E4F0A374642E
:1023FA00F0E4A3F0A3F07F1A7E101210D89002D353
:10240A00E4F0A37434F0A3E4F0A3742EF0A3E4F090
:10241A00A37453F0A3E4F0A37465F0A3E4F0A374E7
:10242A006CF0A3E4F0A37466F0A3E4F0A37454F090
:10243A00A3E4F0A37465F0A3E4F0A37473F0A3E437
:10244A00F0A37474F0E4A3F0A3F07F027E141210D8
:05245A00D81218F72262
:10245F009002D3E4F0A37453F0A3E4F0A37474F0E8
:10246F00A3E4F0A37461F0A3E4F0A37474F0A3E405
:10247F00F0A37475F0A3E4F0A37473F0A3E4F0A3D6
:10248F00743AF0E4A3F0A3F0FFFE1210D89002D339
:10249F00E4F0A37442F0A3E4F0A37449F0A3E4F0D2
:1024AF00A37454F0A3E4F0A37453F0A3E4F0A37463
:1024BF0020F0A3E4F0A37450F0A3E4F0A37445F06C
:1024CF00A3E4F0A37452F0A3E4F0A37420F0A3E408
:1024DF00F0A37454F0A3E4F0A3744FF0A3E4F0A3BB
:1024EF00744EF0A3E4F0A37445F0E4A3F0A3F07FDF
:1024FF00067E1C1210D81218F79002D3E4F0A374C2
:10250F0020F0A3E4F0A37431F0A3E4F0A37435F04A
:10251F00E4A3F0A3F07FD87E0E1210D89002D3E47C
:10252F00F0A37420F0A3E4F0A37420F0A3E4F0A3CD
:10253F007430F0E4A3F0A3F07F707E171210D890E0
:10254F0002D3E4F0A37432F0A3E4F0A37435F0A344
:10255F00E4F0A37436F0E4A3F0A3F07F027E4212FE
:10256F0010D89002D3E4F0A37454F0A3E4F0A37452
:10257F006FF0A3E4F0A3746EF0A3E4F0A37465F01E
:10258F00A3E4F0A37420F0A3E4F0A37430F0A3E469
:10259F00F0A37433F0A3E4F0A37436F0A3E4F0A334
:1025AF007420F0A3E4F0A37428F0A3E4F0A374362E
:1025BF00F0A3E4F0A37435F0A3E4F0A37435F0A313
:1025CF00E4F0A37433F0A3E4F0A37435F0A3E4F0C4
:1025DF00A3744BF0A3E4F0A37448F0A3E4F0A37446
:1025EF007AF0A3E4F0A37429F0A3E4F0A3743AF013
:1025FF00A3E4F0A37420F0A3E4F0A37420F0A3E409
:10260F00F0A37431F0A3E4F0A37436F0A3E4F0A3C5
:10261F007420F0A3E4F0A37462F0A3E4F0A3746950
:10262F00F0A3E4F0A37474F0A3E4F0A37473F0E4E4
:10263F00A3F0A3F07FB67E041210D87F5E7E071240
:0A264F0010D87F067E0A1210D82270
:102659007542027543027544D39000277419F090AE
:102669000027E0FF14F0EF6019AB42E544F92402BA
:10267900F544E543FA3400F543E475F02012BCFF54
:1026890080DDAB42E544F92402F544E543FA340020
:10269900F543E4F5F012BCFF9007FEE024FE700359
:1026A9000227BF1470030228E2147003022A0C24C3
:1026B900036003022B46300203022797300403020A
:1026C9002797300B030227973008030227979002B8
:1026D900D3E4F0A37454F0A3E4F0A37465F0A3E485
:1026E900F0A37473F0A3E4F0A37474F0A3E4F0A36B
:1026F900743FF0A3E4F0A37420F0A3E4F0A37420E2
:10270900F0A3E4F0A37420F0A3E4F0A37420F0A3F1
:10271900E4F0A37420F0A3E4F0A37420F0A3E4F0A0
:10272900A3743CF0A3E4F0A37457F0A3E4F0A374FA
:1027390061F0A3E4F0A37469F0A3E4F0A37474F066
:10274900A3E4F0A37469F0A3E4F0A3746EF0A3E426
:10275900F0A37467F0A3E4F0A37420F0A3E4F0A35A
:102769007445F0A3E4F0A3746EF0A3E4F0A37474C9
:10277900F0A3E4F0A37465F0A3E4F0A37472F0A3EA
:10278900E4F0A3743EF0E4A3F0A3F0022B46900218
:10279900D3E4F0A37454F0A3E4F0A37465F0A3E4C4
:1027A900F0A37473F0A3E4F0A37474F0A3E4F0A3AA
:1027B9007420F0022B4630020302289730040302EA
:1027C9002897300B030228973008030228979002B4
:1027D900D3E4F0A37453F0A3E4F0A37465F0A3E485
:1027E900F0A37474F0A3E4F0A37475F0A3E4F0A368
:1027F9007470F0A3E4F0A3743FF0A3E4F0A3742091
:10280900F0A3E4F0A37420F0A3E4F0A37420F0A3F0
:10281900E4F0A37420F0A3E4F0A37420F0A3E4F09F
:10282900A3743CF0A3E4F0A37457F0A3E4F0A374F9
:1028390061F0A3E4F0A37469F0A3E4F0A37474F065
:10284900A3E4F0A37469F0A3E4F0A3746EF0A3E425
:10285900F0A37467F0A3E4F0A37420F0A3E4F0A359
:102869007445F0A3E4F0A3746EF0A3E4F0A37474C8
:10287900F0A3E4F0A37465F0A3E4F0A37472F0A3E9
:10288900E4F0A3743EF0E4A3F0A3F0022B46900217
:10289900D3E4F0A37416F0A3E4F0A37417F0E4A34F
:1028A900F0A3F07F307E0C1210D89002D3E4F0A38D
:1028B9007453F0A3E4F0A37465F0A3E4F0A3747473
:1028C900F0A3E4F0A37475F0A3E4F0A37470F0A38B
:1028D900E4F0A37420F0022B463002030229BA3037
:1028E90004030229BA300B030229BA30080302296A
:1028F900BA9002D3E4F0A37452F0A3E4F0A3746590
:10290900F0A3E4F0A37463F0A3E4F0A3746FF0A35D
:10291900E4F0A37472F0A3E4F0A37464F0A3E4F008
:10292900A3743FF0A3E4F0A37420F0A3E4F0A3742C
:1029390020F0A3E4F0A37420F0A3E4F0A37420F042
:10294900A3E4F0A3743CF0A3E4F0A37457F0A3E468
:10295900F0A37461F0A3E4F0A37469F0A3E4F0A315
:102969007474F0A3E4F0A37469F0A3E4F0A3746EA3
:10297900F0A3E4F0A37467F0A3E4F0A37420F0A338
:10298900E4F0A37445F0A3E4F0A3746EF0A3E4F0BB
:10299900A37474F0A3E4F0A37465F0A3E4F0A37442
:1029A90072F0A3E4F0A3743EF0E4A3F0A3F0022BC9
:1029B900469002D3E4F0A37416F0A3E4F0A37417CD
:1029C900F0E4A3F0A3F07F187E101210D89002D380
:1029D900E4F0A37452F0A3E4F0A37465F0A3E4F067
:1029E900A37463F0A3E4F0A3746FF0A3E4F0A374F9
:1029F90072F0A3E4F0A37464F0A3E4F0A37420F0EC
:102A0900022B46300203022AE3300403022AE33090
:102A19000B03022AE3300803022AE39002D3E4F00D
:102A2900A37453F0A3E4F0A37465F0A3E4F0A374D2
:062A39006CF0A3E4F0A321
:102A3F007466F0A3E4F0A37420F0A3E4F0A374543D
:102A4F00F0A3E4F0A37465F0A3E4F0A37473F0A310
:102A5F00E4F0A37474F0A3E4F0A3743FF0A3E4F0E4
:102A6F00A37420F0A3E4F0A3743CF0A3E4F0A374E8
:102A7F0057F0A3E4F0A37461F0A3E4F0A37469F03A
:102A8F00A3E4F0A37474F0A3E4F0A37469F0A3E4D7
:102A9F00F0A3746EF0A3E4F0A37467F0A3E4F0A3C3
:102AAF007420F0A3E4F0A37445F0A3E4F0A3746ED4
:102ABF00F0A3E4F0A37474F0A3E4F0A37465F0A39F
:102ACF00E4F0A37472F0A3E4F0A3743EF0E4A3F077
:102ADF00A3F080639002D3E4F0A37416F0A3E4F0A4
:102AEF00A37417F0E4A3F0A3F0FF7E141210D89094
:102AFF0002D3E4F0A37453F0A3E4F0A37465F0A33E
:102B0F00E4F0A3746CF0A3E4F0A37466F0A3E4F014
:102B1F00A37420F0A3E4F0A37454F0A3E4F0A3741F
:102B2F0065F0A3E4F0A37473F0A3E4F0A37474F05E
:0F2B3F00A3E4F0A37420F07F0E7E001210D822C2
:102B4E00300203022C65300403022C65300B0302A5
:102B5E002C65300803022C659007F3E0FFC4540F78
:102B6E00540F75F00AA4FEEF540F2E20E07290025F
:102B7E00D3E4F0A37420F0A3E4F0A37420F0A3E454
:102B8E00F0A37420F0A3E4F0A37420F0A3E4F0A368
:102B9E007420F0A3E4F0A37420F0A3E4F0A3742057
:102BAE00F0A3E4F0A37420F0A3E4F0A37420F0A348
:102BBE00E4F0A37420F0A3E4F0A37420F0A3E4F0F7
:102BCE00A37420F0A3E4F0A37420F0A3E4F0A374A4
:102BDE0020F0A3E4F0A37420F0E4A3F0A3F080703F
:102BEE009002D3E4F0A3743CF0A3E4F0A37457F086
:102BFE00A3E4F0A37461F0A3E4F0A37469F0A3E47A
:102C0E00F0A37474F0A3E4F0A37469F0A3E4F0A34A
:102C1E00746EF0A3E4F0A37467F0A3E4F0A3742041
:102C2E00F0A3E4F0A37445F0A3E4F0A3746EF0A354
:102C3E00E4F0A37474F0A3E4F0A37465F0A3E4F0DD
:102C4E00A37472F0A3E4F0A3743EF0E4A3F0A3F037
:082C5E007F197E001210D8223C
:102C66009002D3E4F0A37420F0A3E4F0A37454F02C
:102C7600A3E4F0A37469F0A3E4F0A37470F0A3E4F2
:102C8600F0A37473F0A3E4F0A3743AF0E4A3F0A302
:102C9600F07F577E031210D89002D3E4F0A374504D
:102CA600F0A3E4F0A37472F0A3E4F0A37465F0A3B8
:102CB600E4F0A37473F0A3E4F0A37473F0A3E4F058
:102CC600A37420F0A3E4F0A37474F0A3E4F0A37457
:102CD60068F0A3E4F0A37465F0A3E4F0A37422F013
:102CE600A3E4F0A37445F0A3E4F0A3746EF0A3E4A8
:102CF600F0A37474F0A3E4F0A37465F0A3E4F0A366
:102D06007472F0A3E4F0A37422F0A3E4F0A3746F4A
:102D1600F0A3E4F0A37472F0A3E4F0A37422F0A38A
:102D2600E4F0A37446F0A3E4F0A37431F0A3E4F056
:102D3600A37422F0E4A3F0A3F07FE07E071210D87C
:102D46009002D3E4F0A37462F0A3E4F0A37475F0E8
:102D5600A3E4F0A37474F0A3E4F0A37474F0A3E402
:102D6600F0A3746FF0A3E4F0A3746EF0A3E4F0A3F1
:102D76007420F0A3E4F0A37474F0A3E4F0A3746FDA
:102D8600F0A3E4F0A37420F0A3E4F0A37473F0A31B
:102D9600E4F0A37474F0A3E4F0A37461F0A3E4F088
:102DA600A37472F0A3E4F0A37474F0A3E4F0A37424
:102DB60020F0A3E4F0A37474F0A3E4F0A37465F028
:102DC600A3E4F0A37473F0A3E4F0A37474F0A3E493
:102DD600F0A3743BF0E4A3F0A3F07FFE7E0A12108A
:102DE600D89002D3E4F0A37455F0A3E4F0A374736F
:102DF600F0A3E4F0A37465F0A3E4F0A37420F0A3B9
:102E0600E4F0A37474F0A3E4F0A37468F0A3E4F010
:102E1600A37465F0A3E4F0A37420F0A3E4F0A37414
:102E260061F0A3E4F0A37472F0A3E4F0A37472F06B
:102E3600A3E4F0A3746FF0A3E4F0A37477F0A3E423
:102E4600F0A37420F0A3E4F0A37426F0A3E4F0A3A7
:102E56007420F0A3E4F0A37422F0A3E4F0A3744575
:102E6600F0A3E4F0A3746EF0A3E4F0A37474F0A3EB
:102E7600E4F0A37465F0A3E4F0A37472F0A3E4F0A5
:102E8600A37422F0E4A3F0A3F07F207E0E1210D8E4
:102E96009002D3E4F0A37462F0A3E4F0A37475F097
:102EA600A3E4F0A37474F0A3E4F0A37474F0A3E4B1
:102EB600F0A3746FF0A3E4F0A3746EF0A3E4F0A3A0
:102EC600742CF0A3E4F0A3746FF0A3E4F0A374727F
:102ED600F0A3E4F0A37420F0A3E4F0A37474F0A3C9
:102EE600E4F0A37468F0A3E4F0A37465F0A3E4F03F
:102EF600A37420F0A3E4F0A37463F0A3E4F0A37436
:102F06006FF0A3E4F0A37472F0A3E4F0A37472F07C
:102F1600A3E4F0A37465F0A3E4F0A37473F0A3E450
:102F2600F0A37470F0A3E4F0A3746FF0A3E4F0A32D
:102F3600746EF0A3E4F0A37464F0A3E4F0A3742D1C
:102F4600F0E4A3F0A3F07F3E7E111210D89002D3D6
:102F5600E4F0A37469F0A3E4F0A3746EF0A3E4F0C4
:102F6600A37467F0A3E4F0A37420F0A3E4F0A374C1
:102F760022F0A3E4F0A37446F0A3E4F0A3746EF089
:102F8600A3E4F0A37422F0A3E4F0A37420F0A3E476
:102F9600F0A37462F0A3E4F0A37475F0A3E4F0A3C5
:102FA6007474F0A3E4F0A37474F0A3E4F0A3746F54
:102FB600F0A3E4F0A3746EF0A3E4F0A37420F0A3EE
:102FC600E4F0A37474F0A3E4F0A3746FF0A3E4F048
:102FD600A37420F0A3E4F0A37473F0A3E4F0A37445
:102FE60065F0A3E4F0A3746CF0A3E4F0A37465F0B9
:102FF600A3E4F0A37463F0A3E4F0A37474F0E4A371
:10300600F0A3F07F5E7E141210D89002D3E4F0A3F2
:103016007474F0A3E4F0A37468F0A3E4F0A37465F9
:10302600F0A3E4F0A37420F0A3E4F0A3746FF0A37C
:10303600E4F0A37474F0A3E4F0A37468F0A3E4F0DE
:06304600A37465F0A3E491
:10304C00F0A37472F0A3E4F0A37420F0A3E4F0A353
:10305C007466F0A3E4F0A37475F0A3E4F0A3746EAB
:10306C00F0A3E4F0A37463F0A3E4F0A37474F0A3EE
:10307C00E4F0A37469F0A3E4F0A3746FF0A3E4F09C
:10308C00A3746EF0A3E4F0A37473F0A3E4F0A37440
:10309C002EF0E4A3F0A3F07F7E7E171210D89002DE
:1030AC00D3E4F0A37442F0A3E4F0A37461F0A3E4BE
:1030BC00F0A37474F0A3E4F0A37474F0A3E4F0A38D
:1030CC007465F0A3E4F0A37472F0A3E4F0A3747934
:1030DC00F0A3E4F0A37420F0A3E4F0A37473F0A3C2
:1030EC00E4F0A37474F0A3E4F0A37461F0A3E4F02F
:1030FC00A37474F0A3E4F0A37475F0A3E4F0A374C8
:10310C0073F0A3E4F0A3743AF0A3E4F0A37420F0FA
:10311C00A3E4F0A37420F0A3E4F0A37420F0A3E4E0
:10312C00F0A37420F0A3E4F0A37420F0A3E4F0A3C4
:10313C007420F0E4A3F0A3F07FDF7E1B1210D812F2
:10314C00A44012A2149007FEE024FD70030231FD8E
:10315C001470030232872402600302330C9002D3F2
:10316C00E4F0A37446F0A3E4F0A37432F0E4A3F00B
:10317C00A3F07FF37E071210D89002D3E4F0A3746F
:10318C0073F0A3E4F0A37465F0A3E4F0A37474F0FB
:10319C00A3E4F0A37420F0A3E4F0A37470F0A3E410
:1031AC00F0A37461F0A3E4F0A37472F0A3E4F0A3B1
:1031BC007461F0A3E4F0A3746DF0A3E4F0A3746560
:1031CC00F0A3E4F0A37474F0A3E4F0A37465F0A38B
:1031DC00E4F0A37472F0A3E4F0A37473F0A3E4F02E
:1031EC00A3743BF0E4A3F0A3F07F087E0B1210D87D
:1031FC00229002D3E4F0A37446F0A3E4F0A374335A
:10320C00F0E4A3F0A3F07FF37E071210D89002D362
:10321C00E4F0A37476F0A3E4F0A37469F0A3E4F0F3
:10322C00A37465F0A3E4F0A37477F0A3E4F0A374A3
:10323C0020F0A3E4F0A37472F0A3E4F0A37465F09F
:10324C00A3E4F0A37463F0A3E4F0A3746FF0A3E41D
:10325C00F0A37472F0A3E4F0A37464F0A3E4F0A3FD
:10326C007473F0A3E4F0A3743BF0E4A3F0A3F0A315
:10327C00F0A3F07F087E0B1210D8229002D3E4F05A
:10328C00A37446F0A3E4F0A37434F0E4A3F0A3F029
:10329C007FF37E071210D89002D3E4F0A37472F07F
:1032AC00A3E4F0A37475F0A3E4F0A3746EF0A3E4AC
:1032BC00F0A37420F0A3E4F0A37473F0A3E4F0A3E0
:1032CC007465F0A3E4F0A3746CF0A3E4F0A374664B
:1032DC00F0A3E4F0A37474F0A3E4F0A37465F0A37A
:1032EC00E4F0A37473F0A3E4F0A37474F0A3E4F01B
:1032FC00A3743BF0E4A3F0A3F07F087E0B1210D86C
:01330C00229E
:01001B0022C2
:10330D001238039002D3E4F0A37420F0A3E4F0A3E9
:10331D007431F0A3E4F0A3742EF0A3E4F0A3744190
:10332D00F0A3E4F0A37444F0A3E4F0A37453F0A36A
:10333D00E4F0A3744CF0A3E4F0A37420F0A3E4F044
:10334D00A37453F0A3E4F0A37474F0A3E4F0A37496
:10335D0061F0A3E4F0A3746EF0A3E4F0A37464F041
:10336D00A3E4F0A37461F0A3E4F0A37472F0A3E4FA
:10337D00F0A37464F0A3E4F0A37473F0A3E4F0A3DA
:10338D00743AF0E4A3F0A3F07FF67E031210D89008
:10339D0002D3E4F0A37420F0A3E4F0A37420F0A30F
:1033AD00E4F0A37418F0A3E4F0A37419F0A3E4F00F
:1033BD00A37441F0A3E4F0A3744EF0A3E4F0A3745E
:1033CD0053F0A3E4F0A37449F0A3E4F0A37420F048
:1033DD00A3E4F0A37454F0A3E4F0A37431F0A3E4D8
:1033ED00F0A3742EF0A3E4F0A37434F0A3E4F0A3DF
:1033FD007431F0A3E4F0A37433F0E4A3F0A3F07FF1
:10340D00167E071210D89002D3E4F0A37420F0A317
:10341D00E4F0A37420F0A3E4F0A37418F0A3E4F097
:10342D00A37419F0A3E4F0A37449F0A3E4F0A3741A
:10343D0054F0A3E4F0A37455F0A3E4F0A37420F0CA
:10344D00A3E4F0A37447F0A3E4F0A3742EF0A3E477
:10345D00F0A37439F0A3E4F0A37439F0A3E4F0A35E
:10346D007432F0A3E4F0A3742EF0A3E4F0A374314E
:10347D00F0A3E4F0A37420F0A3E4F0A37428F0A368
:10348D00E4F0A37447F0A3E4F0A3742EF0A3E4F0EA
:10349D00A37444F0A3E4F0A3744DF0A3E4F0A3747B
:1034AD0054F0A3E4F0A37429F0E4A3F0A3F07F3665
:1034BD007E0A1210D89002D3E4F0A37420F0A3E496
:1034CD00F0A37420F0A3E4F0A37418F0A3E4F0A328
:1034DD007419F0A3E4F0A37449F0A3E4F0A37454B9
:1034ED00F0A3E4F0A37455F0A3E4F0A37420F0A3CB
:1034FD00E4F0A37447F0A3E4F0A3742EF0A3E4F07A
:10350D00A37439F0A3E4F0A37439F0A3E4F0A37429
:10351D0032F0A3E4F0A3742EF0A3E4F0A37432F020
:10352D00A3E4F0A37420F0A3E4F0A37428F0A3E4C3
:10353D00F0A37447F0A3E4F0A3742EF0A3E4F0A37A
:10354D00744CF0A3E4F0A37469F0A3E4F0A37474D5
:10355D00F0A3E4F0A37465F0A3E4F0A37429F0E400
:10356D00A3F0A3F07F567E0D1210D89002D3E4F095
:10357D00A37420F0A3E4F0A37432F0A3E4F0A374D9
:10358D002EF0A3E4F0A37443F0A3E4F0A3746FF062
:10359D00A3E4F0A3746EF0A3E4F0A37474F0A3E4B9
:1035AD00F0A37472F0A3E4F0A37461F0A3E4F0A3AC
:1035BD007473F0A3E4F0A37474F0A3E4F0A3743A6D
:1035CD00F0E4A3F0A3F07F767E101210D89002D312
:1035DD00E4F0A37420F0A3E4F0A37420F0A3E4F0CE
:1035ED00A37420F0A3E4F0A3742DF0A3E4F0A3746E
:1035FD0031F0A3E4F0A37430F0A3E4F0A37420F051
:10360D00A3E4F0A37420F0A3E4F0A37420F0A3E4EA
:10361D00F0A37420F0A3E4F0A37420F0A3E4F0A3CE
:10362D007420F0A3E4F0A37420F0A3E4F0A37430AD
:10363D00F0A3E4F0A37420F0A3E4F0A37420F0A3AE
:10364D00E4F0A37420F0A3E4F0A37420F0A3E4F05D
:10365D00A37420F0A3E4F0A37420F0A3E4F0A3740A
:10366D002BF0A3E4F0A37431F0A3E4F0A37430F0D5
:10367D00E4A3F0A3F07F9E7E151210D89002D3E440
:10368D00F0A37420F0A3E4F0A37433F0A3E4F0A34B
:10369D00742EF0A3E4F0A37442F0A3E4F0A37465D8
:1036AD00F0A3E4F0A37465F0A3E4F0A37470F0A3A9
:1036BD00E4F0A3743AF0A3E4F0A37420F0A3E4F0D3
:1036CD00A37418F0A3E4F0A37419F0A3E4F0A374A9
:1036DD0020F0A3E4F0A3744FF0A3E4F0A3746EF014
:0636ED00A3E4F0A3742029
:1036F300F0A3E4F0A37420F0A3E4F0A37418F0A300
:10370300E4F0A37419F0A3E4F0A37420F0A3E4F0AD
:10371300A3744FF0A3E4F0A37466F0A3E4F0A374DE
:1037230066F0E4A3F0A3F07FBE7E181210D89002D7
:10373300D3E4F0A37420F0A3E4F0A37434F0A3E47F
:10374300F0A3742EF0A3E4F0A37454F0A3E4F0A365
:103753007469F0A3E4F0A3746DF0A3E4F0A37465BB
:10376300F0A3E4F0A37420F0A3E4F0A37453F0A354
:10377300E4F0A37465F0A3E4F0A37474F0A3E4F09D
:10378300A37475F0A3E4F0A37470F0A3E4F0A3743E
:103793003AF0E4A3F0A3F07FDE7E1B1210D8900270
:1037A300D3E4F0A37420F0A3E4F0A37420F0A3E423
:1037B300F0A37414F0A3E4F0A37415F0E4A3F0A34E
:1037C300F0900A17E07002A3E070097F167E0712DB
:1037D30010D88028900A17E07004A3E064017009F0
:1037E3007F367E0A1210D88013900A17E07004A364
:1037F300E0640270077F567E0D1210D8123A6A22D7
:10380300E490002AF0A3F090002AE0FEA3E0FFC3B7
:1038130094B0EE9400501C74542FF582EE340AF5E4
:1038230083E4F090002BE004F0700690002AE0049B
:10383300F080D4E490002AF0A3F090002AE0FEA3E5
:10384300E0FFC3941AEE94005023EF242EFFEE34CE
:103853002AFE7D017C007BB07A0012096E90002B5A
:10386300E004F0700690002AE004F080CDE49000BC
:103873002AF0A3F090002AE0FEA3E0FFC3941AEE1F
:103883009400501C74542FF582EE340AF583E4F04F
:1038930090002BE004F0700690002AE004F080D43E
:1038A300E490002AF0A3F090002AE0FEA3E0FFC317
:1038B30094B0EE940050287C007D2812BBE0EF24E6
:1038C3002EFFEE3403FE7D037B1A7A0012096E90FD
:1038D300002BE004F0700690002AE004F080C82278
:1038E300E490002CF0A3F090002CE0FEA3E0FFC3D3
:1038F300941AEE9400501C74542FF582EE340AF59A
:1039030083E4F090002DE004F0700690002CE004B6
:10391300F080D4E490002CF0A3F090002CE0FEA300
:10392300E0FFC394B0EE940050287C007D2812BBC6
:10393300E0EF242EFFEE3403FE7D037B1A7A0012A0
:10394300096E90002DE004F0700690002CE004F066
:0339530080C82207
:10395600753E02753F1675400B9002D3E4F0A374D2
:1039660020F0A3E4F0A37420F0A3E4F0A37418F00D
:10397600A3E4F0A37419F0E4A3F0A3F07F167E0786
:103986001210D87F367E0A1210D87F567E0D12107E
:10399600D89002D3E4F0A37420F0A3E4F0A374203B
:1039A600F0A3E4F0A37414F0A3E4F0A37415F0E418
:1039B600A3F0A3F09007FDE0B40110E4900A17F01D
:1039C600A3F07F167E071210D8802F9007FDE0B473
:1039D6000211900A17E4F0A304F07F367E0A121053
:1039E600D880179007FDE0B40310900A17E4F0A3FF
:1039F6007402F07F567E0D1210D8900A18E0AB3E86
:083A0600AA3FA94012BBCC222B
:103A0E009002D3E4F0A37420F0A3E4F0A37418F0B2
:103A1E00A3E4F0A37419F0E4A3F0A3F07FC67E181C
:103A2E001210D87FCD7E181210D89002D3E4F0A3D6
:103A3E007420F0A3E4F0A37414F0A3E4F0A37415BF
:103A4E00F0E4A3F0A3F09007DBE060087FCD7E18D2
:0C3A5E001210D8227FC67E181210D82249
:103A6A00753E02753F0A754054E490002EF0A3F0AB
:103A7A0090002EE0FEA3E0FFC3940CEE9400501CCD
:103A8A0074542FF582EE340AF583E4F090002FE0A7
:103A9A0004F0700690002EE004F080D4E490002E2A
:103AAA00F0A3F090002EE0FEA3E0FFC39416EE947C
:103ABA00005023EF2498FFEE343AFE7D017C007B10
:103ACA000C7A0012096E90002FE004F07006900044
:103ADA002EE004F080CDAB3E0540E540AA3F7002DF
:103AEA00053F14F9740F12BBCCE490002EF0A3F03A
:103AFA00C390002FE0941490002EE094005023AB62
:103B0A003E0540E540AA3F7002053F14F974FF12D2
:103B1A00BBCC90002FE004F0700690002EE004F079
:103B2A0080CEAB3E0540E540AA3F7002053F14F93E
:103B3A0074F012BBCC7F987E3A7D037C007B167AA8
:103B4A000012096E7F787E3C12096EE490002EF016
:103B5A00A3F090002EE0FEA3E0FFC3940CEE9400C5
:103B6A00501D74542FF582EE340AF5837408F090D0
:103B7A00002FE004F0700690002EE004F080D37F5E
:103B8A00C07E3A7D017C007B0B7A0012096EE490BC
:103B9A00002EF0A3F090002EE0FEA3E0FFC3940CE9
:103BAA00EE9400501D74542FF582EE340AF5837496
:103BBA0001F090002FE004F0700690002EE004F06F
:103BCA0080D37FCA7E3A7D017C007B0B7A00120982
:103BDA006EE490002EF0A3F090002EE0FEA3E0FF2A
:103BEA00C3940CEE9400501D74542FF582EE340ADF
:103BFA00F5837410F090002FE004F0700690002E08
:103C0A00E004F080D37FD57E3A7D017C007B0B7A7D
:103C1A000012096EE490002EF0A3F090002EE0FE50
:103C2A00A3E0FFC3940BEE9400501D74542FF58249
:103C3A00EE340AF583740FF090002FE004F070065A
:103C4A0090002EE004F080D3900A52E0FF3395E012
:103C5A00FEEF24CAFFEE343AFE7D017C007B0B7A2C
:103C6A000012096E753E02753F0A754054E49000D1
:103C7A002EF0A3F0C390002FE0940B90002EE09456
:103C8A0000503F900A52E0F46015AB3E0540E54013
:103C9A00AA3F7002053F14F974F012BBCC8013AB33
:103CAA003E0540E540AA3F7002053F14F974F1123F
:103CBA00BBCC90002FE004F0700690002EE004F0D8
:103CCA0080B2900A52E0FF3395E0FEEF24CBFFEE7C
:0F3CDA00343AFE7D017C007B0B7A0012096E22CA
:103CE900E4900030F0900030E0FFC3941450147455
:103CF900542FF582E4340AF583E4F0900030E004AF
:103D0900F080E2E4900030F0900030E0FFC3940DC1
:103D1900501BEF24C8FFE4342DFE7D017C007B1489
:103D29007A0012096E900030E004F080DBE4900024
:103D390030F0900030E0FFC39415501BEF24E8FFEA
:103D4900E43430FE7D017C007B147A0012096E9008
:103D59000030E004F080DBE4900030F0900030E0C7
:103D6900FFC39416501BEF2408FFE43434FE7D0191
:103D79007C007B147A0012096E900030E004F08018
:103D8900DBE4900030F0900030E0FFC3940B501B4F
:103D9900EF2427FFE43437FE7D017C007B147A0091
:103DA90012096E900030E004F080DBE4900030F0FE
:103DB900900030E0FFC3940D501BEF249FFFE434C3
:103DC9003FFE7D017C007B147A0012096E90003061
:103DD900E004F080DBE4900030F0900030E0FFC3B5
:103DE900940D501BEF2467FFE43442FE7D017C00F3
:103DF9007B147A0012096E900030E004F080DB1227
:103E09003A0EE4900030F0900030E0FFC394145073
:103E19001574542FF582E4340AF58374FFF0900089
:103E290030E004F080E19007FDE024FE6049146071
:103E390073147003023EDA147003023F071470030F
:103E4900023F6024056003023F8AE4900030F0904D
:103E59000030E0FFC3940D4003023F8AEF24C8FFFE
:103E6900E4342DFE7D017C007B147A0012096E90EA
:103E79000030E004F080D8E4900030F0900030E0A9
:103E8900FFC394154003023F8AEF24E8FFE434306E
:103E9900FE7D017C007B147A0012096E900030E0EF
:103EA90004F080D8E4900030F0900030E0FFC39433
:103EB900164003023F8AEF2408FFE43434FE7D01F3
:103EC9007C007B147A0012096E900030E004F080C7
:103ED900D8E4900030F0900030E0FFC3940B400329
:103EE900023F8AEF2427FFE43437FE7D017C007B03
:103EF900147A0012096E900030E004F080D890071F
:103F0900D8E07029900030F0900030E0FFC39406AB
:103F1900506FEF249FFFE4343FFE7D017C007B144A
:103F29007A0012096E900030E004F080DBE4900022
:103F390030F0900030E0FFC394065045EF24A6FF0F
:103F4900E4343FFE7D017C007B147A0012096E90F7
:103F59000030E004F080DBE4900030F0900030E0C5
:103F6900FFC3940D501BEF2467FFE43442FE7D012B
:103F79007C007B147A0012096E900030E004F08016
:023F8900DB2239
:103F8B008F3E8D3F3078031238037B027A1679000F
:103F9B008B408A41894212BBB1900802F0D394C87E
:103FAB005006E0C394005012E4900033F0900802E6
:103FBB00F0AB40AA41A94212BBCCE53E240AFFE478
:103FCB0033FE900802E0FDFBC3EF9B7480F86E9804
:103FDB005008900033740AF08009C3ED953E0490AD
:103FEB000033F0E4900031F0900033E0FF900031AB
:103FFB00E0FEC39F40030242599002D3E4F0A37446
:10400B0020F0A3E4F0A37420F0E4A3F0A3F0EEFF00
:10401B007E007C027D8012BBE0EF242EFFEE34038A
:10402B00FE1210D8207803024250900031E0FF902E
:10403B000A51E02FFFE433FE1246AC900031E0FF53
:10404B007E007C027D8012BBE0EF2430FFEE340358
:10405B00FE1210D89002D3E4F0A37420F0A3E4F086
:10406B00A37420F0A3E4F0A3742FF0A3E4F0A374E3
:10407B0020F0A3E4F0A37420F0A3E4F0A3742FF0DA
:10408B00A3E4F0A37432F0A3E4F0A37430F0A3E440
:10409B00F0A37420F0A3E4F0A37420F0A3E4F0A346
:1040AB007420F0A3E4F0A37420F0A3E4F0A3742035
:1040BB00F0A3E4F0A3743AF0A3E4F0A37420F0A30C
:1040CB00E4F0A37420F0A3E4F0A3743AF0A3E4F0BB
:1040DB00A37420F0A3E4F0A37420F0E4A3F0A3F006
:1040EB00900031E0FF7E007C027D8012BBE0EF246C
:1040FB0035FFEE3403FE1210D87B027A1679108B43
:10410B00408A418942900031E0253EFFE433FE7C3A
:10411B00017D0E12BBE0E92FF9EA3EFAE924F2F930
:10412B00EA34FFFA8B40F541894212BBB1FFC4540C
:10413B000F75F00AA4FFAB400542E5427002054142
:10414B0014F912BBB1540F2FFF1247DA900031E074
:10415B00FF7E007C027D8012BBE0EF243DFFEE343E
:10416B0003FE1210D8AB40AA41A94212BBB1FFC447
:10417B00540F75F00AA4FF0542E542700205411485
:10418B00F912BBB1540F2FFF1247DA900031E0FF49
:10419B007E007C027D8012BBE0EF2438FFEE3403FF
:1041AB00FE1210D8AB40AA41A94212BBB1FFC454B6
:1041BB000F75F00AA4FF0542E5427002054114F9A0
:1041CB0012BBB1540F2FFF1247DA900031E0FF7E84
:1041DB00007C027D8012BBE0EF2435FFEE3403FE42
:1041EB001210D89000327403F0900032E0C39406A2
:1041FB005053AB40AA41A94212BBB1FFC4540F7537
:10420B00F00AA4FF0542E5427002054114F912BB06
:10421B00B1540F2FFF1247DA900031E0FF7E007C84
:10422B00027D8012BBE0EF2437FDEE3403FCA3E0EC
:10423B0075F003A42DFFE5F03CFE1210D890003270
:10424B00E004F080A4900031E004F0023FF3900210
:10425B00D3E4F0A37411F0E4A3F0A3F0C3E53F950E
:10426B003EFFE49400FE7C027D8012BBE0EF242E27
:10427B00FFEE3403FE1210D8900802E07053900248
:10428B00D3F0A3744EF0A3E4F0A3746FF0A3E4F0A7
:10429B00A37420F0A3E4F0A37472F0A3E4F0A3746E
:1042AB0065F0A3E4F0A37463F0A3E4F0A3746FF0E0
:1042BB00A3E4F0A37472F0A3E4F0A37464F0A3E49A
:1042CB00F0A37421F0E4A3F0A3F07F317E0312106E
:1042DB00D89002D3E4F0A37443F0A3E4F0A3746189
:1042EB00F0A3E4F0A37470F0A3E4F0A37461F0A363
:1042FB00E4F0A37463F0A3E4F0A37469F0A3E4F017
:10430B00A37474F0A3E4F0A37479F0A3E4F0A374A2
:10431B003AF0A3E4F0A37420F0A3E4F0A37432F01A
:10432B00A3E4F0A37430F0A3E4F0A37430F0A3E49F
:10433B00F0A37420F0A3E4F0A37420F0A3E4F0A3A3
:10434B007449F0A3E4F0A3746EF0A3E4F0A374201B
:10435B00F0A3E4F0A37475F0A3E4F0A37473F0A3DB
:06436B00E4F0A37465F00C
:10437100A3E4F0A3743AF0A3E4F0A37420F0A3E45F
:10438100F0A37420F0A3E4F0A37420F0A3E4F0A35D
:104391007420F0A3E4F0A37420F0E4A3F0A3F07F71
:1043A1002E7E1C1210D8900802E0FF7E001246AC4F
:1043B1007F447E1C1210D8900802E0C3946450150B
:1043C1009002D3E4F0A37420F0E4A3F0A3F07F44BF
:0643D1007E1C1210D82230
:1043D700753F027540027541D3C278900035EEF003
:1043E700A3EFF04E7003024651900035E0FEA3E0C4
:1043F700FFC39410EE9427403F7C277D1012BBF437
:10440700AB3FAA40A941E48FF012BCFFAB3FE541A7
:10441700F92402F541E540FA3400F54012BC49FFA2
:10442700AEF07C277D1012BBE0C3900036E09FF012
:10443700900035E09EF08016AB3FE541F92402F588
:1044470041E540FA3400F540E4F5F012BCFF900076
:1044570035E0FEA3E0FFC394E8EE9403403F7C03FE
:104467007DE812BBF4AB3FAA40A941E48FF012BC30
:10447700FFAB3FE541F92402F541E540FA3400F589
:104487004012BC49FFAEF07C037DE812BBE0C3904D
:104497000036E09FF0900035E09EF08016AB3FE5D8
:1044A70041F92402F541E540FA3400F540E4F5F01E
:1044B70012BCFF900035E0FEA3E0FFC39464EE94C6
:1044C70000403F7C007D6412BBF4AB3FAA40A9418A
:1044D700E48FF012BCFFAB3FE541F92402F541E55B
:1044E70040FA3400F54012BC49FFAEF07C007D6411
:1044F70012BBE0C3900036E09FF0900035E09EF0DD
:104507008016AB3FE541F92402F541E540FA340056
:10451700F540E4F5F012BCFF900035E0FEA3E0FFA4
:10452700C3940AEE9400403F7C007D0A12BBF4ABB3
:104537003FAA40A941E48FF012BCFFAB3FE541F928
:104547002402F541E540FA3400F54012BC49FFAEBC
:10455700F07C007D0A12BBE0C3900036E09FF0902C
:104567000035E09EF08016AB3FE541F92402F541A6
:10457700E540FA3400F540E4F5F012BCFF90003650
:10458700E0FFAB3FE541F92402F541E540FA34008D
:10459700F540E48FF012BCFFAB3FE541F924FEF58F
:1045A70041E540FA34FFF540E4F5F012BCFF753FF2
:1045B700027540027541D3E4900034F0900034E076
:1045C700C3940540030246ABAB3FAA40A94112BCC6
:1045D70049FFAEF04E6037D3EF9409EE9400400DDB
:1045E700EF2437FDE43EFCFECFEDCF8007EF24300C
:1045F700FFE43EFEAB3FE541F92402F541E540FA11
:104607003400F540EE8FF012BCFFD278803330785B
:1046170019AB3FE541F92402F541E540FA3400F5CD
:1046270040E475F03012BCFF8017AB3FE541F92439
:1046370002F541E540FA3400F540E475F02012BC7C
:10464700FF900034E004F00245C3E4900034F0909A
:0C4657000034E0C39404501FAB3FE54169
:10466300F92402F541E540FA3400F540E475F02001
:1046730012BCFF900034E004F080D8AB3FE541F971
:104683002402F541E540FA3400F540E475F03012B8
:10469300BCFFAB3FE541F92402F541E540FA3400A4
:0946A300F540E4F5F012BCFF2221
:1046AC007543027544027545D3900037EEF0A3EFC5
:1046BC00F0C39464EE94004052900037E0FEA3E007
:1046CC00FF7C007D6412BBF4EF2430FFE43EFEABB4
:1046DC0043E545F92402F545E544FA3400F544EE8A
:1046EC008FF012BCFF900037E0FAA3E0FB7C007D5A
:1046FC0064FFCEEACE12BBF47C007D6412BBE0C337
:10470C00EB9FF0EA9E900037F08017AB43E545F93C
:10471C002402F545E544FA3400F544E475F0301212
:10472C00BCFF900037E0FEA3E0FFC3940AEE9400B8
:10473C00404A7C007D0A12BBF4EF2430FFE43EFEBD
:10474C00AB43E545F92402F545E544FA3400F5445C
:10475C00EE8FF012BCFF900037E0FAA3E0FB7C0078
:10476C007D0AFFCEEACE12BBF47C007D0A12BBE0C0
:10477C00C3EB9FF0EA9E900037F08017AB43E54502
:10478C00F92402F545E544FA3400F544E475F030BB
:10479C0012BCFF900038E02430FF900037E034006A
:1047AC00FEAB43E545F92402F545E544FA3400F542
:1047BC0044EE8FF012BCFFAB43E545F92402F545FE
:0E47CC00E544FA3400F544E4F5F012BCFF2297
:1047DA007543027544027545D37E00900039EEF0A8
:1047EA00A3EFF0C3940AEE94004052900039E0FE21
:1047FA00A3E0FF7C007D0A12BBF4EF2430FFE43E05
:10480A00FEAB43E545F92402F545E544FA3400F5E3
:10481A0044EE8FF012BCFF900039E0FAA3E0FB7C73
:10482A00007D0AFFCEEACE12BBF47C007D0A12BBE1
:10483A00E0C3EB9FF0EA9E900039F08017AB43E5A6
:10484A0045F92402F545E544FA3400F544E475F0E7
:10485A003012BCFF90003AE02430FF900039E03477
:10486A0000FEAB43E545F92402F545E544FA340078
:10487A00F544EE8FF012BCFFAB43E545F92402F58F
:0F488A0045E544FA3400F544E4F5F012BCFF2292
:104899008F428E418D408C3F7543027544027545A8
:1048A900D3C2787F007E007D007C0012BEB5AF4286
:1048B900AE41AD40AC3F12B8E940067E007F208092
:1048C900047E007F2DAB43E545F92402F545E54417
:1048D900FA3400F544EE8FF012BCFF7F007E007DB4
:1048E900007C0012BEB5AF42AE41AD40AC3F12B83C
:1048F900E9400AAF42AE41AD40AC3F80167FBF7E72
:10490900807D007C0012BEB5AF42AE41AD40AC3FE8
:1049190012B7C290003B12BE677F007E007D007C0B
:104929000012BEB590003B12BE5B12B8E9700302DB
:104939004CBC7F427EC87D007C0012BEB590003B16
:1049490012BE5B12B8E9405F90003B12BE5B12BE1B
:10495900B57F427EC87D007C0012B83A12B976ABA9
:1049690043AA44A945E48FF012BCFFAB43E545F9DE
:104979002402F545E544FA3400F54412BC49FDAC7E
:10498900F0E412B93E12BEB57F427EC87D007C00BC
:1049990012B7C212BEB590003B12BE5B12B6B390FD
:1049A900003B12BE678016AB43E545F92402F54585
:1049B900E544FA3400F544E4F5F012BCFF7F417E8A
:1049C900207D007C0012BEB590003B12BE5B12B880
:1049D900E9405F90003B12BE5B12BEB57F417E206D
:1049E9007D007C0012B83A12B976AB43AA44A945B6
:1049F900E48FF012BCFFAB43E545F92402F545E528
:104A090044FA3400F54412BC49FDACF0E412B93E55
:104A190012BEB57F417E207D007C0012B7C212BE56
:104A2900B590003B12BE5B12B6B390003B12BE6755
:104A39008016AB43E545F92402F545E544FA34000F
:104A4900F544E4F5F012BCFF90003B12BE5B12B9CD
:104A590076AB43AA44A945E48FF012BCFFAB43E50A
:104A690045F92402F545E544FA3400F54412BC49F8
:104A7900FDACF0E412B93E12BEB590003B12BE5B2C
:104A890012B6B390003B12BE67AB43E545F9240269
:104A9900F545E544FA3400F544E475F02E12BCFFFF
:104AA9007F417E207D007C0012BEB590003B12BE86
:044AB9005B12B7C213
:104ABD0012B976AB43E545F92402F545E544FA34E0
:104ACD0000F544E48FF012BCFFAB43E545F9240239
:104ADD00F545E544FA3400F544E4F5F012BCFF7BEE
:104AED00027A0279D58B438A44894512BC49FFAEBF
:104AFD00F04E6021EF2430FFE43EFEAB43E545F977
:104B0D002402F545E544FA3400F544EE8FF012BC6D
:104B1D00FFD2788017AB43E545F92402F545E5440E
:104B2D00FA3400F544E475F02012BCFFAB43AA44FF
:104B3D00A94512BC49FFAEF04E601AEF2430FFE4D8
:104B4D003EFEE5452402F545E43544F544EE8FF08F
:104B5D0012BCFF8033307819AB43E545F92402F5DB
:104B6D0045E544FA3400F544E475F03012BCFF809D
:104B7D0017AB43E545F92402F545E544FA3400F554
:104B8D0044E475F02012BCFFAB43AA44A94512BC06
:104B9D0049FFAEF04E601AEF2430FFE43EFEE545CE
:104BAD002402F545E43544F544EE8FF012BCFF8048
:104BBD0017AB43E545F92402F545E544FA3400F514
:104BCD0044E475F03012BCFF74022545F545E4351B
:104BDD0044F544AB43FAA94512BC492430FFE435F2
:104BED00F0FEE5452402F545E43544F544EE8FF03D
:104BFD0012BCFFAB43E545F92402F545E544FA3413
:104C0D0000F544E4F5F012BCFF7F007E007D007CD2
:104C1D000012BEB5AF42AE41AD40AC3F12B8E94057
:104C2D0003024D457B027A0279D58B438A4489452F
:104C3D0012BC49642045F07039AB43E545F924FEBB
:104C4D00F545E544FA34FFF544E475F02D12BCFF4B
:104C5D00AB43E545F92402F545E544FA3400F54446
:104C6D00E475F02012BCFF74022545F545E435448A
:104C7D00F544AB43AA44A94512BC49642045F060F4
:104C8D0003024D45E54524FEF545E54434FFF54465
:104C9D00E475F02D12BCFFAB43E545F92402F54553
:104CAD00E544FA3400F544E475F02012BCFF22AB64
:104CBD0043E545F92402F545E544FA3400F544E4AD
:104CCD0075F02012BCFFAB43E545F92402F545E52F
:064CDD0044FA3400F54426
:104CE300E475F02012BCFFAB43E545F92402F5451A
:104CF300E544FA3400F544E475F03012BCFFAB43ED
:104D0300E545F92402F545E544FA3400F544E47534
:104D1300F02E12BCFFAB43E545F92402F545E5440B
:104D2300FA3400F544E475F03012BCFFAB43E545BB
:104D3300F92402F545E544FA3400F544E4F5F012AC
:034D4300BCFF2290
:104D46007533027534077535DD75360275370A75A4
:104D5600382E753902753A02753BD3753C02753D9E
:104D660009753EBF9000417414F09002D1E06003D3
:104D7600024EC2AB33AA34A93512BC49FFAEF012BB
:104D860043D77F397E071210D8AB33AA34A93590A2
:104D9600000212BC76FFAEF01243D77F597E0A128C
:104DA60010D8AB33AA34A93590000412BC76FFAEF6
:104DB600F01243D77F797E0D1210D8AB33AA34A9EF
:104DC6003590000612BE031248997F997E10121084
:104DD600D8AB33AA34A93590000A12BE03124899FB
:104DE6007FB97E131210D8AB33AA34A93590000EC2
:104DF60012BE031248997FD97E161210D8AB33AA79
:104E060034A93590001212BC76FFAEF01243D77F5C
:104E1600FB7E191210D8AB36AA37A93812BC49FF47
:104E2600AEF01243D77F4D7E071210D8AB36AA37A5
:104E3600A93890000212BC76FFAEF01243D77F6D00
:104E46007E0A1210D8AB36AA37A93890000412BCD5
:104E560076FFAEF01243D77F8D7E0D1210D8AB369B
:104E6600AA37A93890000612BE031248997FAD7E74
:104E7600101210D8AB36AA37A93890000A12BE0312
:104E86001248997FCD7E131210D8AB36AA37A938AF
:104E960090000E12BE031248997FED7E161210D8AE
:104EA600AB36AA37A93890001212BC76FFAEF012C4
:104EB60043D77F0F7E1A1210D80251679002D1E0B5
:104EC6006402600302515D90003FF090003FE0C332
:104ED60094064003024F72AB3C053EE53EAA3D7088
:104EE60002053D14F912BBB1FF900042E4F0A3EFB6
:104EF600F0AB3C053EE53EAA3D7002053D14F912B5
:104F0600BBB1FE900043E02400F0900042E03EF08A
:104F1600E0FEA3E0FF1243D790003FE014601914AF
:104F2600601F14602514602B146031240570347FD3
:104F36004E7E061210D8802B7F6E7E091210D88006
:104F4600227F8E7E0C1210D880197FAE7E0F121033
:104F5600D880107FCE7E121210D880077FEE7E1585
:104F66001210D890003FE004F0024ED1753C027555
:054F76003D09753EB38A
:104F7B00E490003FF090003FE0C3940640030250E2
:104F8B0021AB3C053EE53EAA3D7002053D14F912EE
:104F9B00BBB1FF900042E4F0A3EFF0AB3C053EE564
:104FAB003EAA3D7002053D14F912BBB1FE900043C1
:104FBB00E02400F0900042E03EF0E0FEA3E0FF12A0
:104FCB0043D790003FE014601914601F1460251440
:104FDB00602B146031240570347F627E061210D86A
:104FEB00802B7F5A7E091210D880227F527E0C12A2
:104FFB0010D880197F4A7E0F1210D880107F427E06
:10500B00121210D880077F3A7E151210D890003FED
:10501B00E004F0024F80900A21E0FFC4540F75F0BA
:10502B000AA4FEEF540F2EFF1247DA7F347E1C12B8
:10503B0010D8900A22E0FFC4540F75F00AA4FEEFBB
:10504B00540F2EFF1247DA7F2F7E1C1210D8900AB6
:10505B0023E0FFC4540F75F00AA4FEEF540F2EFF8C
:10506B001247DA7F2C7E1C1210D89000407403F08C
:10507B00900040E0FFC39406503774212FF582E473
:10508B00340AF583E0FFC4540F75F00AA4FEEF5405
:10509B000F2EFF1247DA900040E075F003A4242E88
:1050AB00FFE5F0341CFE1210D8900040E004F080B5
:1050BB00BF200303025167900E14E0FFC4540F7519
:1050CB00F00AA4FEEF540F2EFF1247DA7FB47E19BD
:1050DB001210D8900E15E0FFC4540F75F00AA4FE01
:1050EB00EF540F2EFF1247DA7FAF7E191210D890B4
:1050FB000E16E0FFC4540F75F00AA4FEEF540F2EEA
:10510B00FF1247DA7FAC7E191210D890004074035F
:10511B00F0900040E0FFC39406504174142FF582C9
:10512B00E4340EF583E0FFC4540F75F00AA4FEEFD0
:10513B00540F2EFF1247DA900040E075F003A424C1
:10514B00AEFFE5F03419FE1210D8900040E004F0E9
:10515B0080BF9002D1E0B4030312516B1254602252
:10516B009002D3E4F0A3740CF0A3E4F0A3740DF05D
:10517B00E4A3F0A3F09009E3E030E7077FE87E07B4
:10518B001210D89009E3E030E6077F087E0B12106F
:10519B00D89009E3E030E5077F287E0E1210D890F7
:1051AB0009E3E030E4077F487E111210D89009E341
:1051BB00E030E3077F687E141210D89009E3E030EB
:1051CB00E2077F887E171210D89009E4E030E707DA
:1051DB007FD47E071210D89009E4E030E6077FF405
:1051EB007E0A1210D89009E4E030E5077F147E0E9A
:1051FB001210D89009E4E030E4077F347E111210CE
:10520B00D89009E4E030E3077F547E141210D89055
:10521B0009E4E030E2077F747E171210D89002D3B6
:10522B00E4F0A3740AF0A3E4F0A3740BF0E4A3F08E
:10523B00A3F09009E3E020E7077FE87E071210D880
:10524B009009E3E020E6077F087E0B1210D8900947
:10525B00E3E020E5077F287E0E1210D89009E3E0EB
:10526B0020E4077F487E111210D89009E3E020E379
:10527B00077F687E141210D89009E3E020E2077FC5
:10528B00887E171210D89009E4E020E7077FD47EC0
:10529B00071210D89009E4E020E6077FF47E0A128B
:1052AB0010D89009E4E020E5077F147E0E1210D889
:1052BB009009E4E020E4077F347E111210D89009A6
:1052CB00E4E020E3077F547E141210D89009E4E049
:1052DB0020E2077F747E171210D89002D3E4F0A35C
:1052EB00741CF0A3E4F0A3741DF0E4A3F0A3F090FE
:1052FB000E1EE030E7077FE57E071210D8900E1EDA
:10530B00E030E6077F057E0B1210D8900E1EE030C2
:10531B00E5077F257E0E1210D8900E1EE030E407B5
:10532B007F457E111210D8900E1EE030E3077F658B
:10533B007E141210D8900E1EE030E2077F857E1788
:10534B001210D89002CBE030E7077FD17E07121006
:10535B00D89002CBE030E6077FF17E0A1210D8908E
:10536B0002CBE030E5077F117E0E1210D89002CBF6
:10537B00E030E4077F317E111210D89002CBE03081
:10538B00E3077F517E141210D89002CBE030E20776
:10539B007F717E171210D89002D3E4F0A37418F02B
:1053AB00A3E4F0A37419F0E4A3F0A3F0900E1EE0B5
:1053BB0020E7077FE57E071210D8900E1EE020E64F
:1053CB00077F057E0B1210D8900E1EE020E5077F9D
:1053DB00257E0E1210D8900E1EE020E4077F457E2E
:1053EB00111210D8900E1EE020E3077F657E141279
:1053FB0010D8900E1EE020E2077F857E171210D882
:10540B009002CBE020E7077FD17E071210D89002E5
:10541B00CBE020E6077FF17E0A1210D89002CBE09A
:10542B0020E5077F117E0E1210D89002CBE020E40E
:10543B00077F317E111210D89002CBE020E3077F5B
:10544B00517E141210D89002CBE020E2077F717EC0
:05545B00171210D82219
:105460007B027A0779DD3003030259ED900804E0EE
:10547000900044F09002D2E0FF70159007DAE0D37C
:105480009410400C9000447422F09002CD740AF005
:10549000EF60159007DAE0D39407400C9000447455
:1054A00022F09002CD740AF0900044E0FF64227074
:1054B000030256CFEF644170030256CF90001412DE
:1054C000BC76FFAEF0E5F06003025A93EF14607013
:1054D0001470030255AA14700302560824036003D3
:1054E000025A939002D3E4F0A37449F0A3E4F0A32A
:1054F0007444F0A3E4F0A3744CF0A3E4F0A3744567
:10550000F0A3E4F0A37420F0A3E4F0A37420F0A3CC
:10551000E4F0A37420F0A3E4F0A37420F0A3E4F07B
:10552000A37420F0A3E4F0A37420F0A3E4F0A37428
:1055300020F0E4A3F0A3F07F08FE1210D8025A93E3
:105540009002D3E4F0A37441F0A3E4F0A37474F0E8
:10555000A3E4F0A37474F0A3E4F0A37465F0A3E4EF
:10556000F0A3746DF0A3E4F0A37470F0A3E4F0A3CF
:105570007474F0A3E4F0A37469F0A3E4F0A3746E70
:10558000F0A3E4F0A37467F0E4A3F0A3F07F08FEB7
:105590001210D8129E29900A2DE0640C6003025A62
:1055A000939007DAE004F0025A939002D3E4F0A358
:1055B0007454F0A3E4F0A37472F0A3E4F0A3746154
:1055C000F0A3E4F0A37469F0A3E4F0A3746EF0A375
:1055D000E4F0A37469F0A3E4F0A3746EF0A3E4F024
:1055E000A37467F0A3E4F0A37420F0A3E4F0A37421
:1055F00020F0E4A3F0A3F07F08FE1210D8129E2939
:10560000E49007DAF0025A939002D3E4F0A37453C3
:10561000F0A3E4F0A37468F0A3E4F0A3746FF0A324
:10562000E4F0A37477F0A3E4F0A37474F0A3E4F0BF
:10563000A37469F0A3E4F0A3746DF0A3E4F0A37481
:1056400065F0A3E4F0A37420F0A3E4F0A37420F0C9
:10565000A3E4F0A37420F0A3E4F0A37420F0A3E487
:10566000F0A37420F0A3E4F0A37420F0A3E4F0A36B
:105670007420F0A3E4F0A37420F0A3E4F0A374205A
:10568000F0A3E4F0A37420F0A3E4F0A37420F0A34B
:10569000E4F0A37420F0A3E4F0A37420F0A3E4F0FA
:1056A000A37420F0A3E4F0A37420F0A3E4F0A374A7
:1056B00020F0E4A3F0A3F07F08FE1210D8900E2093
:1056C000740FF0E49007DAF0900A53F0025A9390C6
:1056D0000044E0642260030258EF9002CDE0C394DE
:1056E0000750141265B27F281201DD126531900255
:1056F000CDE004F0025A9312019912019912019916
:105700007F041201DD120199120199120199900E84
:105710001FE0C3940140030258229002D3E4F0A397
:10572000744FF0A3E4F0A37470F0A3E4F0A37465E5
:10573000F0A3E4F0A3746EF0A3E4F0A37420F0A34C
:10574000E4F0A37466F0A3E4F0A37461F0A3E4F0C2
:10575000A37469F0A3E4F0A3746CF0A3E4F0A37461
:1057600075F0A3E4F0A37472F0A3E4F0A37465F001
:10577000A3E4F0A37421F0A3E4F0A37420F0A3E465
:10578000F0A37428F0A3E4F0A37430F0A3E4F0A332
:105790007478F0A3E4F0A37430F0A3E4F0A37435BC
:1057A000F0A3E4F0A37429F0A3E4F0A37420F0A321
:1057B000E4F0A37420F0A3E4F0A37420F0E4A3F0D9
:1057C000A3F09009E7E0FFC4540F540F900045F098
:1057D000D394094006E02437FE8007900045E0247A
:1057E00030FEEEFD9002F5E4F0A3EDF0EF540F90E3
:1057F0000045F0D394094006E02437FF800790006D
:1058000045E02430FF9002F7E4F0A3EFF07F087E3C
:10581000001210D8E4900E20F09002D274FFF00233
:1058200058D09002D3E4F0A37441F0A3E4F0A37441
:1058300063F0A3E4F0A37474F0A3E4F0A37469F03C
:06584000A3E4F0A374765E
:10584600F0A3E4F0A37461F0A3E4F0A37474F0A3EE
:10585600E4F0A37469F0A3E4F0A3746FF0A3E4F09A
:10586600A3746EF0A3E4F0A37420F0A3E4F0A37491
:1058760074F0A3E4F0A37469F0A3E4F0A3746DF0EC
:10588600A3E4F0A37465F0A3E4F0A3746FF0A3E4BB
:10589600F0A37475F0A3E4F0A37474F0A3E4F0A38A
:1058A6007421F0A3E4F0A37420F0A3E4F0A3742021
:1058B600F0A3E4F0A37420F0A3E4F0A37420F0E4D2
:1058C600A3F0A3F07F08FE1210D8900E1FE0C39439
:1058D600055006E004F0025A93E49007DAF0900EC1
:1058E6001FF09002CDF0025A939002D3E4F0A37415
:1058F6004CF0A3E4F0A3746FF0A3E4F0A37473F088
:10590600A3E4F0A37473F0A3E4F0A37420F0A3E47B
:10591600F0A3746FF0A3E4F0A37466F0A3E4F0A31D
:105926007420F0A3E4F0A37473F0A3E4F0A3746905
:10593600F0A3E4F0A37467F0A3E4F0A3746EF0A3FD
:10594600E4F0A37461F0A3E4F0A3746CF0A3E4F0B4
:10595600A37421F0A3E4F0A37421F0A3E4F0A374EC
:1059660020F0A3E4F0A37420F0A3E4F0A37420F0E5
:10597600A3E4F0A37420F0E4A3F0A3F07F08FE12E2
:1059860010D8E4900E20F0900A53E0C394FA500326
:10599600E004F0900A53E0D394145003025A93D2D1
:1059A600071265B27F051201DDD204D20C900A2DD2
:1059B6007401F0C20AE4900E1EF09002CBF012655C
:1059C60031120159E49002CEF0900A53F0900E2065
:1059D600F09007DAF09002D2F0900E1FF09002CD10
:1059E600F012A1C0025A939002D3E4F0A37452F0CD
:1059F600A3E4F0A37465F0A3E4F0A37463F0A3E456
:105A0600F0A3746FF0A3E4F0A37472F0A3E4F0A320
:105A16007464F0A3E4F0A37420F0A3E4F0A3744E3E
:105A2600F0A3E4F0A3746FF0A3E4F0A3742EF0E403
:105A3600A3F0A3F07F08FE1210D8900E23E0FF7E9D
:105A4600001246AC7F127E001210D89002D3E4F00A
:105A5600A37450F0A3E4F0A37461F0A3E4F0A3747C
:105A660067F0A3E4F0A37465F0A3E4F0A37420F058
:105A76009002D1E024319002DEF0E4339002DDF0B2
:105A8600E49002DFF0A3F07F16FE1210D820031177
:105A9600900A17E0FFA3E0900046CFF0A3EFF08056
:105AA6003A7B027A1679108B3F8A408941900E2301
:105AB600E0FF7E007C017D0E12BBE0E92FF9EA3E95
:105AC600FAE924F8F9EA34FFFA8B3FF540894112E6
:105AD600BBB1FF900046E4F0A3EFF0900046E0FE75
:105AE600A3E0FFEE6003025BD0EF605324FE700379
:105AF600025B8B046003025BD09002D3E4F0A374D4
:105B06003CF0A3E4F0A37447F0A3E4F0A3742EF0F2
:105B1600A3E4F0A37444F0A3E4F0A3744DF0A3E46B
:105B2600F0A37454F0A3E4F0A3743EF0A3E4F0A34E
:105B36007420F0E4A3F0A3F07F20FE1210D8229088
:105B460002D3E4F0A3743CF0A3E4F0A37441F0A301
:105B5600E4F0A3744EF0A3E4F0A37453F0A3E4F0CE
:105B6600A37449F0A3E4F0A3743EF0A3E4F0A37495
:105B760020F0A3E4F0A37420F0E4A3F0A3F07F20C8
:105B8600FE1210D8229002D3E4F0A3743CF0A3E4F2
:105B9600F0A37447F0A3E4F0A3742EF0A3E4F0A3FB
:105BA600744CF0A3E4F0A37469F0A3E4F0A3747456
:105BB600F0A3E4F0A37465F0A3E4F0A3743EF0E46C
:0B5BC600A3F0A3F07F20FE1210D822F5
:105BD1009007F9E0FFC4540F540F75F00AA4FEEFCB
:105BE100540F2EFF1247DA7F347E1F1210D8900710
:105BF100F7E0FFC4540F540F75F00AA4FEEF540FE1
:105C01002EFF1247DA7F2F7E1F1210D89007F6E081
:105C1100FFC4540F540F75F00AA4FEEF540F2EFF6A
:105C21001247DA7F2C7E1F1210D89007F5E0FFC4CF
:105C3100540F540F75F00AA4FEEF540F2EFF1247B4
:105C4100DA7F237E1F1210D89007F4E0FFC4540FAF
:105C5100540F75F00AA4FEEF540F2EFF1247DA7F9E
:105C6100267E1F1210D89007F3E0FFC4540F540F83
:105C710075F00AA4FEEF540F2EFF1247DA7F297E3A
:105C81001F1210D89007F8E0B407004003025E85A8
:105C9100905C98F8282873025CAD025CF1025D35D6
:105CA100025D79025DBD025E01025E449002D3E4B1
:105CB100F0A37453F0A3E4F0A37475F0A3E4F0A38C
:105CC100746EF0A3E4F0A37464F0A3E4F0A3746130
:105CD100F0A3E4F0A37479F0A3E4F0A37420F0A39B
:105CE100E4F0A37420F0A3E4F0A37420F0025E8535
:105CF1009002D3E4F0A3744DF0A3E4F0A3746FF029
:105D0100A3E4F0A3746EF0A3E4F0A37464F0A3E43D
:105D1100F0A37461F0A3E4F0A37479F0A3E4F0A319
:105D21007420F0A3E4F0A37420F0A3E4F0A37420A2
:105D3100F0025E859002D3E4F0A37454F0A3E4F082
:105D4100A37475F0A3E4F0A37465F0A3E4F0A37465
:105D510073F0A3E4F0A37464F0A3E4F0A37461F01E
:105D6100A3E4F0A37479F0A3E4F0A37420F0A3E416
:105D7100F0A37420F0025E859002D3E4F0A374577F
:105D8100F0A3E4F0A37465F0A3E4F0A37464F0A3BA
:105D9100E4F0A3746EF0A3E4F0A37465F0A3E4F05F
:105DA100A37473F0A3E4F0A37464F0A3E4F0A37408
:105DB10061F0A3E4F0A37479F0025E859002D3E46C
:105DC100F0A37454F0A3E4F0A37468F0A3E4F0A387
:105DD1007475F0A3E4F0A37472F0A3E4F0A37473F8
:105DE100F0A3E4F0A37464F0A3E4F0A37461F0A35E
:105DF100E4F0A37479F0A3E4F0A37420F0025E85CB
:105E01009002D3E4F0A37446F0A3E4F0A37472F01B
:105E1100A3E4F0A37469F0A3E4F0A37464F0A3E431
:105E2100F0A37461F0A3E4F0A37479F0A3E4F0A308
:105E31007420F0A3E4F0A37420F0A3E4F0A3742091
:105E4100F080419002D3E4F0A37453F0A3E4F0A3F3
:105E51007461F0A3E4F0A37474F0A3E4F0A3747587
:105E6100F0A3E4F0A37472F0A3E4F0A37464F0A3CC
:105E7100E4F0A37461F0A3E4F0A37479F0A3E4F077
:105E8100A37420F0E49002E5F0A3F07F377E1F12A7
:035E910010D82204
:105E94007533027534077535DD75360275370A7545
:105EA400382E9000487402F0A3E4F0C27830030363
:105EB400025F5D753902753AF2F53B900048F0A334
:105EC400F0900048E0FEA3E0FFC3EE9402502EAB36
:105ED40039053BE53BAA3A7002053A14F912BBB105
:105EE400FD74032FF582EE3408F583EDF09000493C
:105EF400E004F07006900048E004F080C4900903C8
:105F0400E0900052F0642060359000487401F0A3E2
:105F1400E4F0900048E0FEA3E0FFC394E4EE9401B3
:105F2400501C74032FF582EE3408F583E4F09000DE
:105F340049E004F07006900048E004F080D4900931
:105F4400E3E054FC7006A3E054FC60089007D374AB
:105F54000FF08005E49007D3F09002D1E0600302D3
:105F640064159009A6E0FE9009A5E07C002400FFDA
:105F7400EC3EAB33AA34A9358FF012BCFF9009AACA
:105F8400E0FE9009A9E02400FFEC3EAB36AA37A955
:105F9400388FF012BCFF9009A4E0FE9009A3E0241E
:105FA40000FFEC3EAB33AA34A9359000028FF01207
:105FB400BD209009A8E0FE9009A7E02400FFEC3E74
:105FC400AB36AA37A9389000028FF012BD20900991
:105FD4000CE0FE90090BE02400FFEC3EAB33AA3446
:105FE400A9359000128FF012BD20900914E0FE90A4
:105FF4000913E02400FFEC3EAB36AA37A938900021
:10600400128FF012BD20AB33AA34A93590001212BE
:10601400BC76FDACF04C70030261FFE412B93E1291
:10602400BEB57F427EC87D007C0012B83A90004A1B
:1060340012BE67AB33AA34A93512BC49FDACF04C8F
:106044006018E412B93E12BEB590004A12BE5B124B
:10605400B83A90004E12BE678025AB33AA34A935F6
:1060640090000212BC76FDACF0E412B93E12BEB54B
:1060740090004A12BE5B12B83A90004E12BE67906E
:10608400004E12BE5B12B976EF7805CEC313CE1361
:10609400D8F97805C333CE33CED8F9FFAB33AA345D
:1060A400A935900004EE8FF012BD2090000412BCBC
:1060B40076FFAEF012BC496F7003EE65F0601DAB65
:1060C40033AA34A93590000212BC76FFAEF09000DA
:1060D4000412BC766F7003E5F06E7022AB33AA3401
:1060E400A93590001212BC76646445F07003026214
:1060F4000E900004E475F02012BCB002620EAB33C3
:10610400AA34A935900004740275F00012BCB09052
:10611400000412BC76D39400E5F094204011AB3314
:10612400AA34A935900004742075F00012BD20AB88
:0561340033AA34A93577
:1061390012BC49FDACF04C6057E412B93E12BEB531
:10614900AB33AA34A93590000412BC76FDACF0E457
:1061590012B93E12B83A90004A12BE677F427EC811
:106169007D007C0012BEB590004A12BE5B12B7C218
:1061790090004E12BE6790004E12BE5B12B976AB0C
:1061890033AA34A935900012EE8FF012BD20807524
:10619900AB33AA34A93590000212BC76FDACF0E409
:1061A90012B93E12BEB5AB33AA34A9359000041218
:1061B900BC76FDACF0E412B93E12B83A90004A122E
:1061C900BE677F427EC87D007C0012BEB590004A42
:1061D90012BE5B12B7C290004E12BE6790004E12FB
:1061E900BE5B12B976AB33AA34A935900012EE8F93
:1061F900F012BD20800FAB33AA34A935900004E416
:10620900F5F012BD20AB36AA37A93890001212BC9E
:1062190076FDACF04C7003026322E412B93E12BE63
:10622900B57F427EC87D007C0012B83A90004A12C0
:10623900BE67AB36AA37A93812BC49FDACF04C6031
:1062490018E412B93E12BEB590004A12BE5B12B8EC
:106259003A90004E12BE678025AB36AA37A938900E
:10626900000212BC76FDACF0E412B93E12BEB59044
:10627900004A12BE5B12B83A90004E12BE679000F7
:106289004E12BE5B12B976EF7805CEC313CE13D882
:10629900F97805C333CE33CED8F9FFAB36AA37A97F
:1062A90038900004EE8FF012BD2090000412BC76E5
:1062B900FFAEF012BC496F7003EE65F0601DAB369E
:1062C900AA37A93890000212BC76FFAEF0900004FC
:1062D90012BC766F7003E5F06E701CAB36AA37A955
:1062E9003890001212BC76646445F0600A9000048C
:1062F900E475F02012BCB0AB36AA37A93890000477
:1063090012BC76D39400E5F09404401C9000047408
:106319000475F00012BD20800FAB36AA37A938905A
:106329000004E4F5F012BD2090090DE0FF9000543F
:10633900F0FC12B94212BEB57F407E007D007C00A0
:1063490012B83AAB33AA34A93590000612BE35907B
:106359000915E0FF900054F0FC12B94212BEB57F56
:10636900407E007D007C0012B83AAB36AA37A938C6
:1063790090000612BE35900916E0FF900054F0FC1B
:1063890012B94212BEB57F407E007D007C0012B872
:106399003AAB33AA34A93590000A12BE3590090EDA
:1063A900E0FF900054F0FC12B94212BEB57F407E66
:1063B900007D007C0012B83AAB36AA37A9389000A4
:1063C9000A12BE3590090FE0FCE412B94212BEB5BB
:1063D9007F407E007D007C0012B83AAB33AA34A915
:1063E9003590000E12BE35900917E0FCE412B9424F
:1063F90012BEB57F407E007D007C0012B83AAB36F4
:10640900AA37A93890000E12BE35802320032090A8
:106419000E1EE0FF9009E3E0FEEF4E900E1EF09095
:1064290002CBE0FF9009E4E0FEEF4E9002CBF09042
:106439000052E0FF24F8602124F8603024F0605A0B
:1064490024206003026519AB33AA34A935900014DE
:10645900E4F5F012BD20026528AB33AA34A93590C2
:106469000014E475F00112BD20026528AB33AA348B
:10647900A935900014E475F00212BD209007D9E007
:106489006F70030265283003030265281201999091
:106499000A2D7401F0C20A026528AB33AA34A93562
:1064A900900014E475F00312BD209007D9E0FF9025
:1064B9000052E06F60692003661201BB7F0112017F
:1064C900DD1201BB7F011201DD1201BBE490005313
:1064D900F0900053E0C39405502CE0FF24F3F582BB
:1064E900E43407F583E0FEEFFDC374059DFDE494F4
:1064F90000FC74212DF582EC340AF583EEF090004E
:1065090053E004F080CB9007F9E0900A21F0800F66
:10651900AB33AA34A935900014E4F5F012BD2090EC
:086529000052E09007D9F022B6
:10653100C27890F24A7401F0A3E4F0A3F090F3FD65
:106541007415F0D207C278E4900055F0A3F0C3901F
:106551000056E09430900055E09475502B90F20273
:10656100E020E004D27880209000577432F090004F
:1065710057E0FF14F0EF70F6900056E004F070065B
:10658100900055E004F080C630781A900A17E07048
:1065910004A3E06402600790F2007403F02290F219
:1065A100007407F0221201BB7F011201DD1201BB51
:0165B10022C7
:1065B200C278300766E4900058F0A3F0C390005907
:1065C200E09430900058E09475502B90F202E02055
:1065D200E004D278802090005A740AF090005AE0C9
:1065E200FF14F0EF70F6900059E004F0700690008E
:1065F20058E004F080C6900903E0B4200890F2004D
:10660200740EF0800690F2007404F07F141201DD23
:0E66120090F2007404F07F141201DDC2072222
:10662000C27890F24A7401F0A3E4F0A3F090F3FD75
:106630007415F0D207E490005BF0A3F0C390005C07
:10664000E0943090005BE09475502B90F202E020D3
:10665000E004D278802090005D7432F090005DE01C
:10666000FE14F0EE70F690005CE004F0700690000E
:106670005BE004F080C6307821EF24FE600E1460E9
:10668000122402702090F2007401F02290F2007443
:1066900002F02290F200740FF0221201BB7F01126F
:0666A00001DD1201BB2226
:1066A600900E1AE054F8F04403F090F800F0E490ED
:1066B600005EF090005EE0C39464501D900E1AE0F8
:1066C60054FEF090F800F04401900E1AF090F80095
:1066D600F090005EE004F080DA900E1AE054F8F0D4
:1066E6004401F090F800F0E490005EF0900A52E069
:1066F600FF3395E0FE7C007D0312BBE0EF2423FF11
:10670600E43EFE90005EE0C39FEE6480F8748098DD
:10671600501D900E1AE054FEF090F800F0440190DF
:106726000E1AF090F800F090005EE004F080BD9044
:0B6736000E1AE04407F090F800F0227B
:10674100200223200B2020081D20041A900A29E48E
:10675100F0A304F0900A4804F0A304F0A37405F038
:10676100A304F00267F3200209200B06200803307E
:10677100041F20031C200119200D16900A29E4F0A2
:10678100A37402F0900A4814F0A3F0A3F0A3F080E0
:1067910061300B19300316900A29E4F0A37403F059
:1067A100900A4814F0A3F0A3F0A3F0804530041E32
:1067B10030011B900A29E4F0A37404F0900A487494
:1067C10002F0A304F0A37405F0A304F08024300BBD
:1067D1001A300D17900A29E4F0A37405F0900A48C5
:1067E1007402F0A3F0A3F0A3F08007E4900A29F06B
:0667F100A3F01209B4221E
:1067F70020021F200B1C200819200416900A2BE4E6
:10680700F0A304F0900A4804F0E4A3F0A3F0A3F087
:106817008049300B2120031E200D1B900802E060E9
:1068270015900A2BE4F0A37402F0900A48F0A3F045
:10683700A3F0A3F0802530041B200118900A2BE455
:10684700F0A37403F0900A48F0E4A3F0A3F0A37454
:0F68570004F08007E4900A2BF0A3F01209B4229A
:1068660020021C200B19200816200413900A46E467
:10687600F0A304F0A304F0A3F0A3F0A3F0806E301D
:106886000B23200320900802E0601A200D17900ABF
:1068960046E4F0A37402F0A304F0E4A3F0A3F0A38B
:1068A6007404F0804830041C200119900A46E4F074
:1068B600A37404F0A37402F0A304F0A37405F0A378
:1068C60004F0802930021F9007FDE0B40618900AF4
:1068D60046E4F0A37403F0A314F0E4A3F0A3740455
:1068E600F0A304F08007E4900A46F0A3F01209B47E
:0168F600227F
:1068F700200222200B1F20081C200419900A4EE4B6
:10690700F0A304F0900A4804F0E4A3F0A3F0A3F086
:10691700D2080269D0300B23200320200D1D9008D8
:1069270002E06017900A4EE4F0A37402F0900A4860
:10693700F0E4A3F0A3F0A3F00269D030041E200115
:106947001B900A4EE4F0A37406F0900A487402F014
:10695700A304F0A37405F0A304F0806D30041D3088
:10696700011A900A4EE4F0A37403F0900A4814F059
:10697700A304F0A37405F0A304F0804D300B1E3080
:106987000D1B200318900A4EE4F0A37404F0900A3C
:10699700487402F0E4A3F0A3F0A3F0802C300222A5
:1069A7009007FDE0B4061B900A4EE4F0A37405F0CF
:1069B700900A487402F0E4A3F0A37404F0A304F06F
:0D69C7008007E4900A4EF0A3F01209B422FC
:1069D400200212200B0F20080C200409900A15E451
:1069E400F0A304F02230020A900A15E4F0A3740222
:1069F400F022300B1020030D200D0A900A15E4F04C
:106A0400A37403F02230040D20010A900A15E4F067
:106A1400A37405F022300B0D30030A900A15E4F03C
:0D6A2400A37405F022E4900A15F0A3F022FF
:106A3100200212200B0F20080C2004099007D4E437
:106A4100F0A304F02230020A9007D4E4F0A3740208
:106A5100F022300B1020030D200D0A9007D4E4F032
:106A6100A37403F02230040D20010A9007D4E4F04E
:106A7100A37405F022300B0D30030A9007D4E4F023
:0D6A8100A37405F022E49007D4F0A3F022E6
:106A8E003002109007FDE0B404099002CFE4F0A3A9
:106A9E0004F0223002119007FDE0B4050A9002CFF7
:106AAE00E4F0A37405F0223002119007FDE0B40665
:106ABE000A9002CFE4F0A37402F022200403300BFC
:106ACE00119002D1E0B4010A9002CFE4F0A3740356
:106ADE00F022300B1020030D200D0A9002CFE4F0AF
:0D6AEE00A37404F022E49002CFF0A3F02284
:106AFB003002109007FDE0B40409900E21E4F0A3DE
:106B0B0004F0223002119007FDE0B4050A900E212B
:106B1B00E4F0A37405F0223002119007FDE0B406F7
:106B2B000A900E21E4F0A37402F022200403300B30
:106B3B00119002D1E0B4010A900E21E4F0A374038A
:106B4B00F022300B1020030D200D0A900E21E4F0E3
:0D6B5B00A37404F022E4900E21F0A3F022B8
:106B6800200270200B6D20086A200467900A4CE40C
:106B7800F0A304F09007FEE024FE602214603114B4
:106B8800603F24036003026C61900A487402F0A31A
:106B980004F0A37405F0A304F0D204026C61900A17
:106BA800487402F0E4A3F0A3F0A3F0D202026C61EF
:106BB800900A487402F0A3F0A3F0A3F0D20B026C81
:106BC80061900A487402F0E4A3F0A3F0A3F0D2089D
:106BD800026C613002149007FDE0C39405500B90DD
:106BE8000A4CE4F0A37402F0806F300B23200320DA
:106BF800200D1D900802E06017900A4CE4F0A37481
:106C080003F0900A4814F0E4A3F0A3F0A3F080493D
:106C18003002129007FDE0B4050B900A4CE4F0A393
:106C28007406F080343002129007FDE0B4060B9031
:106C38000A4CE4F0A37404F0801F2004033003120C
:106C48009002D1E0B4010B900A4CE4F0A37405F073
:0D6C58008007E4900A4CF0A3F01209B4226A
:03000300026C6527
:106C6500C0E0C083C082C0D075D0087EFCE4FDEDD5
:106C7500C394FF50040F0D80F6E4FD7D037830E4E6
:106C8500F608DDFC7D03E59054F064F07003026DB9
:106C95004FE4FDEDC39403502CED70048E908008F5
:106CA500EE25E04402FEF590E4FFEFC39432500375
:106CB5000F80F7E590C4540F540FFC74302DF8C6BF
:106CC500ECC60D80CE7590F0C200E4900A50F0FD40
:106CD500EDC39403505974302DF8E6FE640F604CF3
:106CE500EE24F5601924FE60241460302407703901
:106CF500ED25E025E004900A50F0D200802BED252B
:106D0500E025E02402900A50F0D200801CED25E039
:106D150025E02403900A50F0D200800DED25E025F2
:106D2500E02404900A50F0D2002000030D80A1E574
:106D35009054F064F070F8E4FDEDC394C850040F6E
:106D45000D80F6E59054F0B4F0F9D0D0D082D08320
:036D5500D0E03259
:03002300026D5813
:106D5800C0E0C0F0C083C082C0D075D008C2AF30D8
:106D68009837E599603120022E20082B200428202E
:106D78000B25B43A0B1201999007FB740FF080179A
:106D8800B439089007FB741FF0800CB4380912015D
:106D9800999007FB742FF0C298D2AFD0D0D082D090
:066DA80083D0F0D0E032C0
:106DAE0075330275341675350075360275371675DE
:106DBE003810AB33AA34A93512BBB1FF7E007C016B
:106DCE007D0E12BBE0E41CFD90006412BE67C299FA
:106DDE00D28EE490005FF090005FE0C394145015E3
:106DEE00742BA2D0929BF5993099FDC29990005FB9
:106DFE00E004F080E2AB33AA34A93512BBB1A2D0C5
:106E0E00929BF5993099FDC29990006012BE730065
:106E1E0000000090006412BE5B12BEB590006012BE
:106E2E00BE5B12BDDE504EAB36AA37A93812BBB1CF
:106E3E00A2D0929BF5993099FDC29974012538F52F
:106E4E0038E43537F537E490005FF090005FE0C32B
:106E5E0094C85005E004F080F290006012BE5B1200
:106E6E00BEB57F017E007D007C0012BD4F9000609C
:106E7E0012BE67809EE490005FF090005FE0C394C6
:106E8E00145017C299740AA2D0929BF5993099FDAD
:0B6E9E00C29990005FE004F080E02249
:106EA900C299D28E7439A2D0929BF5993099FDC2BC
:026EB90099221C
:106EBB0078697C007D027B057AA679687E007F1954
:106ECB0012BB7FD28EE4900068F0900068E0FFC3A5
:106EDB0094165020C29974692FF582E43400F5831F
:106EEB00E0A2D0929BF5993099FDC299900068E091
:056EFB0004F080D62226
:106F0000C200900A50E0B40B005054906F12F82861
:106F10002873026F33026F37026F3B026F3F026FBD
:106F200043026F47026F4B026F4F026F53026F575E
:106F3000026F5B1201BB221274412212739922125A
:106F400070F322126F6322127D8E22127C24221291
:106F5000783722127A1922127EE1221281EB221254
:036F600001BB2250
:106F6300126741900A29E0FEA3E0FFEE600302707E
:106F7300EFEF70030270EB24FE70030270091470CC
:106F8300030270871470030270B91470030270C493
:106F9300240460030270EF1201999007FE7401F05C
:106FA300D204D20C900A2DF0C20A900E20E0704D4C
:106FB300900082F0900082E0C39405502CE0FF24FF
:106FC300F3F582E43407F583E0FEEFFDC374059D1A
:106FD300FDE49400FC74212DF582EC340AF583EE74
:106FE300F0900082E004F080CB9007F9E0900A2152
:106FF300F0E4900E1EF09002CBF0126531120159AD
:10700300E49002CEF022120199C204E49007D8F072
:10701300C208C20BC2029007FD04F0E49002D1F053
:10702300900A5104F0900E23F09007FF7480F03023
:107033000931C209E4900082F0900082E0C3940811
:107043005021E0FF2419F582E4340AF583E0FE744D
:10705300F32FF582E43407F583EEF0900082E00429
:10706300F080D6120159900E20E070031265B2E44D
:107073009002CEF0900A28F09002CDF09007DAF05B
:1070830012A21422120199C203E49002D1F09007D4
:10709300FF7480F01202741203741209B412220AEC
:1070A300120FC1122659900A51E0FF900E23E0FD02
:1070B300D278123F8B22120199C201D20C120159CC
:1070C30022120199C20D12027412037412220A12BF
:1070D3000FC11226591209B4900A51E0FF900E23F2
:1070E300E0FDD278123F8B221201BB221201BB2298
:1070F3001267F7900A2BE0FEA3E0FFEE6003027332
:1071030095EF24FE60251470030273652402600367
:107113000273951201999007FE7402F0D202120FC6
:10712300C112265912330D123CE92212019990081B
:1071330002E0FF7003027398900E23E0FEC39401F4
:107143005003027398EE6F70707B027A16F98B33DB
:107153008A34F535900802E014F0E012BBCCEED38C
:1071630094014006900E23E014F0E4900083F0A312
:10717300F0C3900084E0940A900083E094004003FD
:10718300027355900A51E0FFD39401401CEF240988
:10719300FFE433FE900E23E0FDD3EF9D7480F86E81
:1071A300984006900A51E014F0900084E004F070D7
:1071B30006900083E004F080B87B027A1679008B96
:1071C300338A348935900802E014F0E012BBCC1204
:1071D30038039002D3E4F0A37444F0A3E4F0A3745F
:1071E30065F0A3E4F0A3746CF0A3E4F0A37465F07A
:1071F300A3E4F0A37474F0A3E4F0A37469F0A3E42C
:10720300F0A3746EF0A3E4F0A37467F0A3E4F0A317
:107213007420F0A3E4F0A37472F0A3E4F0A3746504
:10722300F0A3E4F0A37463F0A3E4F0A3746FF0A3FA
:10723300E4F0A37472F0A3E4F0A37464F0A3E4F0A5
:10724300A3742EF0A3E4F0A3742EF0A3E4F0A374CC
:107253002EF0E4A3F0A3F07F207E0E1210D87B0261
:107263007A1679108B338A348935900E23E024FF04
:10727300FFE434FFFE7C017D0E12BBE0E92FF9EA47
:107283003E8B33F534893579108B368A378938E06C
:10729300FF7E0012BBE0E92FF9EA3E8B36F5378912
:1072A30038E4900083F0A3F0900E23E0FF900802EF
:1072B300E0C39FFFE49400CF2401CF3400FE7C01A0
:1072C3007D0E12BBE0C3900084E09F900083E09E9C
:1072D3005034AB360538E538AA377002053714F950
:1072E30012BBB1FFAB330535E535AA347002053463
:1072F30014F9EF12BBCC900084E004F07006900008
:1073030083E004F080A2E4900083F0A3F0C3900034
:1073130084E0940A900083E094005036900A51E090
:10732300FFD39401401CEF2409FFE433FE900E23A6
:10733300E0FDD3EF9D7480F86E984006900A51E00B
:1073430014F0900084E004F07006900083E004F0F1
:1073530080BB900A51E0FF900E23E0FDD278123FEC
:107363008B22120199D2017B027A1679008B338A20
:1073730034893512BBB1900802F01209B4900802A7
:10738300E0C394C85006E4FF1288BF227F0212882C
:06739300BF221201BB2223
:10739900126866900A46E0FEA3E0FFEE60030274FD
:1073A9003DEF24FE603014603B14603F240360030A
:1073B90002743D120199C2029007FE7403F0D20BC8
:1073C900120FC1122659900A51E0FF900E23E0FDD9
:1073D900D278123F8B22120199D20D1209B47F0182
:1073E9001288BF221201991292BE22120199D20764
:1073F9001265B27F051201DDD204D20C900A2D74F8
:1074090001F0C20AE4900E1EF09002CBF012653131
:10741900120159E49002CEF0900A53F0900E20F038
:107429009007DAF09002D2F0900E1FF09002CDF0A2
:0874390012A1C0221201BB22C6
:107441007536027537097538031268F7900A4EE0F0
:10745100FEA3E0FFEE6003027833EF24FE603514F3
:1074610070030275ED1470030277B1147003027793
:10747100F9147003027800240560030278331201C5
:10748100999007FE7404F0120FC11226591209B423
:10749100129549221201997536027537097538031B
:1074A1007B027A1679108B338A348935900E23E06A
:1074B10024FFFFE434FFFE7C017D0E12BBE0E92FC7
:1074C100F9EA3E8B33F5348935E4900085F0A3F079
:1074D100C3900086E0940E900085E094015034AB97
:1074E100330535E535AA347002053414F912BBB100
:1074F100FFAB360538E538AA377002053714F9EFC6
:1075010012BBCC900086E004F07006900085E00488
:10751100F080BD74FF2538F53874FF3537F53774C1
:10752100FF2538F53874FF3537F537E4900085F0DD
:10753100A3F0900085E0FEA3E0FFC39406EE940063
:107541005035AB36E5381538AA3770021537F912C0
:10755100BBB1FDC374059FFFE49EFE74212FF5822C
:10756100EE340AF583EDF0900086E004F0700690A9
:107571000085E004F080BB74FF2538F53874FF35D1
:1075810037F537E4900085F0A3F0900085E0FEA385
:10759100E0FFC39406EE94005035AB36E53815385C
:1075A100AA3770021537F912BBB1FDC374059FFFED
:1075B100E49EFE74142FF582EE340EF583EDF09007
:1075C1000086E004F07006900085E004F080BB9036
:1075D10009CBE0900E1EF09009CCE09002CBF0D2E6
:1075E10003D20CE49002D1F01201592212019990B8
:1075F1000802E0C394C8400374C7F07B027A16798D
:10760100108B338A348935900802E0FF7E007C01BB
:107611007D0E12BBE0E92FF9EA3E8B33F534893553
:107621008B36753709753803E4900085F0A3F0C3F4
:10763100900085E094015034AB360538E538AA371F
:107641007002053714F912BBB1FFAB330535E535CF
:10765100AA347002053414F9EF12BBCC900086E015
:1076610004F07006900085E004F080C39007F9E013
:10767100FFAB330535E535AA347002053414F9EF53
:1076810012BBCCE4900085F0A3F0900085E0FEA34E
:10769100E0FFC39405EE94005036C374049FFFE4E9
:1076A1009EFE74F32FF582EE3407F583E0FFAB33D2
:1076B1000535E535AA347002053414F9EF12BBCC57
:0376C100900086B0
:1076C400E004F07006900085E004F080BA900A1897
:1076D400E0FFAB330535E535AA347002053414F9FF
:1076E400EF12BBCCE4900085F0A3F0C3900086E0D9
:1076F4009406900085E09400502FA3E02421F582A5
:10770400E4340AF583E0FFAB330535E535AA34707C
:1077140002053414F9EF12BBCC900086E004F0703B
:1077240006900085E004F080C27B027A1679108B03
:10773400338A348935900802E0FF7E007C017D0E97
:1077440012BBE0E92FF9EA3EFAE924C8F9E43A8BDE
:1077540033F5348935900E1EE0FFAB330535E5353E
:10776400AA347002053414F9EF12BBCC9002CBE0BA
:10777400FFAB330535E535AA347002053414F9EF4F
:1077840012BBCC900802E004F0E0D394C840037428
:10779400C8F07B027A1679008B338A3489359008D5
:1077A40002E012BBCCC201D20C120159221201997F
:1077B400C202D20BC20D900A517401F0900E23F054
:1077C400E4900802F07B027A16F98B368A37F53892
:1077D40012BBCC12027412037412220A120FC112C9
:1077E40026591209B4900A51E0FF900E23E0FDD20D
:1077F40078123F8B221201991293F92212019912E5
:1078040001591265B2E4900E20F09002CEF0900A75
:1078140028F09002D2F0900E1FF09002CDF0900765
:10782400DAF0900E1EF09002CBF0900A53F0221280
:0378340001BB2273
:107837001269D4900A15E0FEA3E0FFEE6003027A16
:1078470015EF24FE60421470030279891470030255
:1078570079711470030279F024046003027A151217
:1078670001999007FEE0D394014005E014F08006EB
:107877009007FE7404F0C2021238E3120FC11226F9
:1078870059122C6612001B221201999007FDE0D3B2
:1078970094014005E014F080069007FD7406F0900F
:1078A70007FDE064066003027956D209900087F06D
:1078B700900087E0C394085021E0FF24F3F582E4A9
:1078C7003407F583E0FE74192FF582E4340AF58353
:1078D700EEF0900087E004F080D69000897402F003
:1078E700900089E0C394045074E4900088F09000FD
:1078F70088E0C394085050E4900087F0900087E038
:10790700FFC39412501574542FF582E4340AF5839B
:1079170074FFF0900087E004F080E1900089E07543
:10792700F00AA42489FFE5F03449FE900088E07C42
:10793700002FFFEC3EFE7D017B127A0012096E904C
:107947000088E004F080A7900089E004F08091C2ED
:1079570009D206129079E4900A4AF0A3F0126866F9
:107967001268F71209B4123CE9221201999007FF35
:10797700E0C394F45005E0240AF0229007FF74FE58
:10798700F022120199900A51E0FF900E23E0D39F55
:107997004007E014F0C205803EEFD39401402CE489
:1079A700900087F0900087E0C3940A5014900A5122
:1079B700E0D394014003E014F0900087E004F080E6
:1079C700E3900E23E014F0D205800C900E2374018F
:1079D700F0900A51F0D205900A51E0FF900E23E093
:1079E700FDA2059278123F8B221201999002D1E0F5
:1079F700D394004005E014F080069002D17403F0A0
:107A07009002D1E064016002D20C120159221201E6
:027A1700BB2290
:107A1900126A319007D4E0FEA3E0FFEE6003027C16
:107A290020EF24FE6042147003027B6B1470030282
:107A39007B53147003027BFC24046003027C201234
:107A490001999007FEE0C394045005E004F0800614
:107A59009007FE7401F0C2021238E3120FC1122618
:107A690059122C6612001B221201999007FDE0C3DE
:107A790094065005E004F080069007FD7401F0902B
:107A890007FDE064066003027B38D20990008AF0A2
:107A990090008AE0C394085021E0FF24F3F582E4C2
:107AA9003407F583E0FE74192FF582E4340AF5836F
:107AB900EEF090008AE004F080D690008C7402F019
:107AC90090008CE0C394045074E490008BF0900013
:107AD9008BE0C394085050E490008AF090008AE04B
:107AE900FFC39412501574542FF582E4340AF583B8
:107AF90074FFF090008AE004F080E190008CE0755A
:107B0900F00AA42489FFE5F03449FE90008BE07C5B
:107B1900002FFFEC3EFE7D017B127A0012096E9068
:107B2900008BE004F080A790008CE004F08091C203
:107B390009D206129079E4900A4AF0A3F012686615
:107B49001268F71209B4123CE9221201999007FF51
:107B5900E0D3940B4005E024F6F0229007FF74016E
:107B6900F022120199900A51E0FF2409FDE433FC47
:107B7900900E23E0F9C39DEC6480F874809850144A
:107B8900900802E0FEE9C39E500A900E23E004F03B
:107B9900C2058041EFC394C85031900802E0FFE963
:107BA900C39F5027900A51E0C394BE500EE0240AA7
:107BB900F0900E23E004F0D205801A900E23E00421
:107BC900F0900A51E004F0D205800A900802E09092
:107BD9000E23F0D205900E23E0C3940150037401E3
:107BE900F0900A51E0FF900E23E0FDA20592781271
:107BF9003F8B221201999002D1E0C394035005E012
:107C090004F08005E49002D1F09002D1E0640160B3
:0B7C190002D20C120159221201BB2202
:107C2400126A8E9002CFE0FEA3E0FFEE6003027DB5
:107C34008AEF24FE603F147003027CE61470030292
:107C44007D18147003027CCB24046003027D8A90A7
:107C54000A52E0D364809476400B120199900A5240
:107C6400E014F080091201BB900A5274F6F0123A43
:107C74006A1266A6221201999007FCE0FF700304C1
:107C8400F022EFB401079007FC7402F022EFB40273
:107C9400079007FC7405F022EFB40306E49007FC98
:107CA400F022EFB404079007FC7403F022EFB4054C
:107CB400079007FC7406F022EF64066003027D8DD2
:107CC4009007FC7404F0221201999007D8E0D39431
:107CD400004005E014F080069007D87401F0123CCF
:107CE400E9221201999007DCE070149007FFE0D3B9
:107CF40094024004E014F0229007FF74FEF02290F6
:107D040007FFE0D3940B4005E024F6F0229007FF30
:107D14007401F022120199E490008DF090008DE03E
:107D2400C3940A5014900E23E0D394014003E0144A
:107D3400F090008DE004F080E3900A51E0FF900E93
:107D440023E0C39F501890008DE0FF14F0EF600E05
:107D5400900A51E0D3940140EDE014F080E8900ED5
:107D640023E0C3940150037401F0900A51E0C394DA
:107D74000150037401F0900A51E0FF900E23E0FDDE
:0A7D8400D278123F8B221201BB22BD
:107D8E00126AFB900E21E0FEA3E0FFEE6003027E7E
:107D9E00DDEF24FE603F147003027E501470030268
:107DAE007E82147003027E3624046003027EDD9010
:107DBE000A52E0C36480948A500B120199900A52C1
:107DCE00E004F080091201BB900A52740AF0123AD4
:107DDE006A1266A6221201999007FCE0FF700474E5
:107DEE0003F022EFB40106E49007FCF022EFB40298
:107DFE00079007FC7401F022EFB403079007FC74A0
:107E0E0004F022EFB404079007FC7406F022EFB4DE
:107E1E0005079007FC7402F022EF64066003027EF1
:107E2E00E09007FC7405F0221201999007D8E0C388
:107E3E0094015005E004F08005E49007D8F0123C60
:107E4E00E9221201999007DCE070149007FFE0C35D
:107E5E0094FE5004E004F0229007FF7401F022908B
:107E6E0007FFE0C394F45005E0240AF0229007FFC8
:107E7E0074FEF022120199E490008EF090008EE0D4
:107E8E00C3940A5018900802E0FF900E23E0C39F9F
:107E9E005003E004F090008EE004F080DF900A5171
:107EAE00E0FF900E23E0C39FD39409401290008E02
:107EBE00E0FF14F0EF6008900A51E004F080EE90BD
:107ECE000A51E0FF900E23E0FDD278123F8B221272
:037EDE0001BB22C3
:107EE100753602753709753803753902753A167595
:107EF1003B08126B68900A4CE0FEA3E0FFEE6003C2
:107F01000281E7EF24FE70030280001470030280F7
:107F11003214700302818A1470030281DD1470032C
:107F21000281B1240560030281E7120199122659E9
:107F31009007FEE024FE7003027FC8147003027FE5
:107F4100D2147003027FF0240360030281EA9007D8
:107F5100FE7401F0D204D20C900A2DF0C20A900EE8
:107F610020E0705A90008FF0A3F090008FE0FEA304
:107F7100E0FFC39405EE94005030E024F3F582E471
:107F81003407F583E0FDC374059FFFE49EFE742171
:107F91002FF582EE340AF583EDF0900090E004F0C5
:107FA100700690008FE004F080C09007F9E0900A1D
:107FB10021F0E4900E1EF09002CBF0126531120117
:107FC10059E49002CEF0221209B412330D123CE9A9
:107FD10022C2029007FE7403F0120FC112265990BB
:107FE1000A51E0FF900E23E0FDD278123F8B2290E0
:107FF10007FE7404F0120FC112265912954922127C
:1080010001999007FDE024FE6011146012146013C1
:10801100240360030281EA123956221239562212D0
:10802100395622900A52E0AB39AA3AA93B12BBCC8D
:10803100221201997536027537097538037B027A68
:108041001679108B338A348935900E23E024FFFF93
:10805100E434FFFE7C017D0E12BBE0E92FF9EA3E1C
:108061008B33F5348935E490008FF0A3F0C3900091
:1080710090E0940E90008FE094015034AB330535BD
:10808100E535AA347002053414F912BBB1FFAB36E1
:108091000538E538AA377002053714F9EF12BBCC61
:1080A100900090E004F0700690008FE004F080BD35
:1080B10074FF2538F53874FF3537F53774FF2538E7
:1080C100F53874FF3537F537E490008FF0A3F09061
:1080D100008FE0FEA3E0FFC39406EE94005035ABA1
:1080E10036E5381538AA3770021537F912BBB1FDDC
:1080F100C374059FFFE49EFE74212FF582EE340ABE
:10810100F583EDF0900090E004F0700690008FE0B0
:1081110004F080BB74FF2538F53874FF3537F53727
:10812100E490008FF0A3F090008FE0FEA3E0FFC386
:108131009406EE94005035AB36E5381538AA377001
:10814100021537F912BBB1FDC374059FFFE49EFE12
:1081510074142FF582EE340EF583EDF0900090E06B
:1081610004F0700690008FE004F080BB9009CBE032
:0E817100900E1EF09009CCE09002CBF0D203ED
:10817F00D20CE49002D1F012015922120199C209D6
:10818F009007FD7401F0D206129079E4900A4AF03C
:10819F00A3F01268661268F71209B4123CE9128D47
:1081AF00E4229007D8E070069007DBF08006900776
:1081BF00DB74FFF07B027A1679098B338A348935A9
:1081CF009007DBE012BBCC120199123CE92212019D
:0C81DF00999007DCE0F4F0221201BB22B2
:1081EB00120199900E1DE0F4F0600B900A27E04409
:1081FB000890F1FCF022900A27E054F790F1FCF084
:01820B002250
:10820C008F3C8E3B8D3A8C397F077E007D007C0045
:10821C0012BEB5AF3CAE3BAD3AAC3912BDAC900022
:10822C0095EFF0AF3CAE3BAD3AAC3912BEB57F40EA
:10823C007E017D007C0012BD6212BED4900093EED4
:10824C00F0A3EFF0AF3CAE3BAD3AAC3912BEB57F0C
:10825C00087E007D007C0012BD6212BED412BEB539
:10826C007F287E007D007C0012BD6212BEDC900077
:10827C0096EFF0FB900093E0FEA3E0FF7C007D28DE
:10828C0012BBE0EB2F900098F0EC3E900097F0E4DE
:10829C00900091F0A3F0900091E0FEA3E0FFC39456
:1082AC0080EE9402501C74542FF582EE340AF58340
:1082BC00E4F0900092E004F07006900091E004F07D
:1082CC0080D4900097E0FEA3E0FF7D037C007B80D0
:1082DC007A0212096E900095E0F9C39402400302F1
:1082EC0083ABE4900099F0900099E0C39410502D6A
:1082FC00E0FF90A82193FE900095E004FDEEC8ED00
:10830C00C8088002C313D8FCFE74542FF582E434E1
:10831C000AF583EEF0900099E004F080CA90009882
:10832C00E024FFFF900097E034FFFE7D017C007B92
:10833C00107A0012096EE4900099F0900099E0C355
:10834C0094105047E0FF90A82193FE900095E0FD1B
:10835C00C374079DFCEEC8ECC8088002C333D8FC7C
:10836C00FEEF90A83193FCED04FDECC8EDC808803D
:10837C0002C313D8FC4EFE74542FF582E4340AF574
:10838C0083EEF0900099E004F080B0900097E0FE4E
:10839C00A3E0FF7D017C007B107A0012096E22E9BC
:1083AC00C3940640030284C9E4900099F0900099AC
:1083BC00E0C39410502DE0FF90A82193FE900095FF
:1083CC00E004FDEEC8EDC8088002C313D8FCFE74AF
:1083DC00542FF582E4340AF583EEF0900099E00412
:1083EC00F080CA900098E024FFFF900097E034FFE3
:1083FC00FE7D017C007B107A0012096EE4900099DE
:10840C00F0900099E0C394105047E0FF90A821939E
:10841C00FE900095E0FDC374079DFCEEC8ECC80807
:10842C008002C333D8FCFEEF90A83193FCED04FD21
:10843C00ECC8EDC8088002C313D8FC4EFE74542F50
:10844C00F582E4340AF583EEF0900099E004F080B4
:10845C00B0900097E0FEA3E0FF7D017C007B107ADA
:10846C000012096EE4900099F0900099E0C394100A
:10847C005031E0FF90A83193FE900095E0FDC3745D
:10848C00079DFDEEC8EDC8088002C333D8FCFE740E
:10849C00542FF582E4340AF583EEF0900099E00451
:1084AC00F080C6900098E02401FF900097E0340023
:1084BC00FE7D017C007B107A0012096E22E4900094
:1084CC0099F0900099E0C394105047E0FF90A821D8
:1084DC0093FE900095E0FDC374079DFCEEC8ECC8BC
:1084EC00088002C333D8FCFEEF90A83193FCED0456
:1084FC00FDECC8EDC8088002C313D8FC4EFE7454C2
:10850C002FF582E4340AF583EEF0900099E004F044
:10851C0080B0900097E0FEA3E0FF7D017C007B1013
:10852C007A0012096EE4900099F0900099E0C394DF
:10853C00105031E0FF90A83193FE900095E0FDC300
:10854C0074079DFDEEC8EDC8088002C333D8FCFE4D
:10855C0074542FF582E4340AF583EEF0900099E020
:10856C0004F080C6900098E02401FF900097E0345E
:0E857C0000FE7D017C007B107A0012096E2249
:10858A0075330275340975351B75360275370A75E8
:10859A003854753902753A00753B9A2003079009D9
:1085AA0003E0B42002C20CE490019AF090019AE030
:1085BA00C394805050AB33AA34A93512BBB1FFC45F
:1085CA00540F540FFFAB39053BE53BAA3A7002053D
:1085DA003A14F9EF12BBCCAB330535E535AA347042
:1085EA0002053414F912BBB1540FFFAB39053BE550
:1085FA003BAA3A7002053A14F9EF12BBCC90019AE1
:10860A00E004F080A7E490019CF090019CE0C39400
:10861A002040030286F9E490019BF090019BE0FF61
:10862A00C39440501474542FF582E4340AF583E459
:10863A00F090019BE004F080E2E490019AF090014E
:10864A009AE0C3940840030286DC75360275370A3D
:10865A00753854E4A3F090019AE0FF90019CE0750C
:10866A00F008A42FF582E435F0F583E582249AF523
:10867A0082E5833400F583E075F004A4FF90019B42
:10868A00E0C39FE5F06480F8748098503CAB36AA4A
:10869A0037A93812BBB1FF90019AE0FEC374079E56
:1086AA00FE7401C8EEC8088002C333D8FC4FFFAB82
:1086BA00360538E538AA377002053714F9EF12BBC8
:1086CA00CC90019BE004F0808D90019AE004F002C6
:1086DA00864890019CE0242CFFE43440FEE4FDFC33
:1086EA007B40FA12096E90019CE004F00286142283
:1086FA0075330275340975351B7536027537017580
:10870A00389DE490029DF090029DE0C39480505001
:10871A00AB33AA34A93512BBB1FFC4540F540FFFAF
:10872A00AB360538E538AA377002053714F9EF1267
:10873A00BBCCAB330535E535AA347002053414F9E0
:10874A0012BBB1540FFFAB360538E538AA377002B1
:10875A00053714F9EF12BBCC90029DE004F080A714
:10876A009007FFE0FF7E001246AC7FBB7E0412102A
:10877A00D89007FFE02401FFE433FE1246AC7F6382
:10878A007E071210D89007FFE02402FFE433FE129E
:10879A0046AC7F0B7E0A1210D89007FFE0249CF5A6
:1087AA0082E43401F583E0FF1247DA7FCC7E0412BB
:1087BA0010D89007FFE0249DF582E43401F583E0A8
:1087CA00FF1247DA7F747E071210D89007FFE02461
:1087DA009EF582E43401F583E0FF1247DA7F1C7EBE
:1087EA000A1210D89007FFE024FFFDE434FFFCE4EE
:1087FA0012B93E12BEB57F407E8A7D007C0012B758
:10880A00C290029F12BE6790029F12BE5B12B97697
:10881A001243D77FC07E041210D89007FFE0FD7C78
:10882A0000E412B93E12BEB57F407E8A7D007C000C
:10883A0012B7C290029F12BE6790029F12BE5B12CD
:10884A00B9761243D77F687E071210D89007FFE0E7
:10885A002401FDE433FCE412B93E12BEB57F407E2A
:10886A008A7D007C0012B7C290029F12BE679002F6
:10887A009F12BE5B12B9761243D77F107E0A12107E
:10888A00D89007FFE0FF5407FE90029EF0FDEF1319
:10889A001313541F2454FFE43419FEEF7803C3332F
:1088AA00CE33CED8F97C002DFFEC3EFEE4FD1282D9
:0588BA000C12546022C5
:1088BF008F39753A02753B0A753C54753D02753E0A
:1088CF0002753FD3E49002A3F0A3F0C39002A4E09B
:1088DF0094209002A3E094005022AB3A053CE53C73
:1088EF00AA3B7002053B14F9E412BBCC9002A4E042
:1088FF0004F070069002A3E004F080CFE49002A38E
:10890F00F0A3F09002A3E0FEA3E0FFC3942EEE9439
:10891F000050287C007D2812BBE0EF2460FFEE346E
:10892F0033FE7D037B1F7A0012096E9002A4E004D0
:10893F00F070069002A3E004F080C8753A02753B10
:10894F000A753C54E49002A3F0A3F0C39002A4E094
:10895F00941A9002A3E094005023AB3A053CE53CF7
:10896F00AA3B7002053B14F974FF12BBCC9002A412
:10897F00E004F070069002A3E004F080CEE49002D1
:10898F00A3F0A3F09002A3E0FEA3E0FFC39429EEAF
:10899F00940050287C007D2812BBE0EF2460FFEE8E
:1089AF003433FE7D037B1A7A0012096E9002A4E025
:1089BF0004F070069002A3E004F080C87FF17E39C6
:1089CF007D037C007B1A7A0012096E7F197E3A12A2
:1089DF00096E7F417E3A12096E753A02753B0A7530
:1089EF003C54E49002A3F0A3F0C39002A4E09424BB
:1089FF009002A3E094005023AB3A053CE53CAA3B20
:108A0F007002053B14F9747012BBCC9002A4E00401
:108A1F00F070069002A3E004F080CEAB3A053CE57F
:108A2F003CAA3B7002053B14F974F012BBCCAB3A75
:108A3F00053CE53CAA3B7002053B14F974F012BBF0
:108A4F00CCAB3A053CE53CAA3B7002053B14F974EC
:108A5F00F012BBCC7F6A7E347D017C007B277A00CD
:108A6F0012096E753A02753B0A753C54E49002A3E5
:108A7F00F0A3F0C39002A4E0941C9002A3E0940032
:108A8F005022AB3A053CE53CAA3B7002053B14F97A
:108A9F00E412BBCC9002A4E004F070069002A3E0B5
:108AAF0004F080CFE49002A3F0A3F09002A3E0FEC5
:108ABF00A3E0FFC3942EEE940050287C007D281273
:108ACF00BBE0EF2460FFEE340CFE7D037B1C7A00CD
:108ADF0012096E9002A4E004F070069002A3E00465
:108AEF00F080C8E539147003028BCA147003028C2E
:108AFF0088147003028D2D24036003028DE390020E
:108B0F00D3E4F0A37453F0A3E4F0A37461F0A3E4EF
:108B1F00F0A37476F0A3E4F0A37465F0A3E4F0A3DC
:108B2F007420F0A3E4F0A37474F0A3E4F0A3746FC3
:108B3F00F0A3E4F0A37420F0A3E4F0A3744EF0A329
:108B4F00E4F0A3746FF0A3E4F0A3742EF0A3E4F0A9
:108B5F00A37420F0A3E4F0A37420F0A3E4F0A374B3
:108B6F0020F0A3E4F0A3742CF0A3E4F0A37459F065
:108B7F00A3E4F0A37465F0A3E4F0A37473F0A3E48B
:108B8F00F0A3742FF0A3E4F0A3744EF0A3E4F0A3CA
:108B9F00746FF0A3E4F0A3743FF0E4A3F0A3F07FAD
:108BAF006A7E0E1210D8900802E02401FFE433FE13
:108BBF001246AC7F757E0E1210D8229002D3E4F0CD
:108BCF00A37443F0A3E4F0A3746CF0A3E4F0A374D4
:108BDF0065F0A3E4F0A37461F0A3E4F0A37472F062
:108BEF00A3E4F0A37420F0A3E4F0A37461F0A3E472
:108BFF00F0A3746CF0A3E4F0A3746CF0A3E4F0A3FF
:108C0F007420F0A3E4F0A37472F0A3E4F0A37465EE
:108C1F00F0A3E4F0A37463F0A3E4F0A3746FF0A3E4
:108C2F00E4F0A37472F0A3E4F0A37464F0A3E4F08F
:108C3F00A37473F0A3E4F0A3742CF0A3E4F0A37473
:108C4F0059F0A3E4F0A37465F0A3E4F0A37473F0F8
:108C5F00A3E4F0A3742FF0A3E4F0A3744EF0A3E405
:108C6F00F0A3746FF0A3E4F0A3743FF0E4A3F0A3B8
:108C7F00F07F697E0E1210D8221201BB9002D3E44E
:108C8F00F0A37443F0A3E4F0A3746FF0A3E4F0A394
:068C9F007476F0A3E4F07E
:108CA500A37465F0A3E4F0A37472F0A3E4F0A374D5
:108CB50020F0A3E4F0A3744EF0A3E4F0A3746FF0E6
:108CC500A3E4F0A3742EF0A3E4F0A37432F0A3E4BC
:108CD500F0A37430F0A3E4F0A37430F0A3E4F0A3A0
:108CE5007420F0A3E4F0A3742CF0A3E4F0A374596A
:108CF500F0A3E4F0A37465F0A3E4F0A37473F0A308
:108D0500E4F0A3742FF0A3E4F0A3744EF0A3E4F011
:108D1500A3746FF0A3E4F0A3743FF0E4A3F0A3F011
:108D25007F697E0E1210D8229002D3E4F0A374530B
:108D3500F0A3E4F0A37465F0A3E4F0A3746EF0A3CC
:108D4500E4F0A37464F0A3E4F0A37469F0A3E4F081
:108D5500A3746EF0A3E4F0A37467F0A3E4F0A37426
:108D650020F0A3E4F0A37472F0A3E4F0A37465F01B
:108D7500A3E4F0A37463F0A3E4F0A3746FF0A3E499
:108D8500F0A37472F0A3E4F0A37464F0A3E4F0A379
:108D95007473F0A3E4F0A37420F0A3E4F0A3742E9D
:108DA500F0A3E4F0A3742EF0A3E4F0A3742EF0A3D3
:108DB500E4F0A3742EF0A3E4F0A3742EF0A3E4F082
:108DC500A3742EF0A3E4F0A3742EF0A3E4F0A3742F
:0F8DD5002EF0E4A3F0A3F07F697E0E1210D822D7
:108DE4009002CC740FF07B027A16790A12BBCC90F5
:108DF4000E1AE054E7F090F800F0E49002A5F09029
:108E040002A5E0C3940A500F900E1AE04410F090AB
:108E140002A5E004F080E8900E1AE090F800F090CB
:108E240002A7E4F0A3748EF0E49002A5F09002A5EA
:108E3400E0C3940850339002A7E0FEA3E0FF30E0C3
:108E440003D38001C39290EEC3139002A7F0EF13F3
:108E5400A3F0900E1AE0FF441890F800F0EF54F7D6
:108E6400F09002A5E004F080C4E49002A7F0A3F01F
:108E74009002A5F09002A5E0C3940850339002A795
:108E8400E0FEA3E0FF30E003D38001C39290EEC381
:108E9400139002A7F0EF13A3F0900E1AE0FF44180A
:108EA40090F800F0EF54F7F09002A5E004F080C4CD
:108EB400900E1AE054E790F800F07F021201DD9062
:108EC4000E1AE04410F090F800F09002A7E4F0A32A
:108ED40074BEF0E49002A5F09002A5E0C39408509B
:108EE400339002A7E0FEA3E0FF30E003D38001C388
:108EF4009290EEC3139002A7F0EF13A3F0900E1A12
:108F0400E0FF441890F800F0EF54F7F09002A5E069
:108F140004F080C4E49002A5F09002A5E0FFC3949D
:108F240008505B74F32FF582E43407F583E0FF9077
:108F340002A7E4F0A3EFF0E49002A6F09002A6E00A
:108F4400C394085031A3E0FEA3E0FF30E003D380D4
:108F540001C39290EEC3139002A7F0EF13A3F09015
:108F64000E1AE0FF441890F800F0EF54F7F0900266
:108F7400A6E004F080C69002A5E004F0809B900E69
:0A8F84001AE054E7F090F800F02224
:108F8E00C2AF900E1AE054E7F090F800F0E49002B1
:108F9E00A9F09002A9E0C3940A5005E004F080F213
:108FAE00900E1AE04410F090F800F09002ABE4F04E
:108FBE00A374BFF0E49002A9F09002A9E0C3940854
:108FCE0050339002ABE0FEA3E0FF30E003D380010C
:108FDE00C39290EEC3139002ABF0EF13A3F0900E7A
:108FEE001AE0FF441890F800F0EF54F7F09002A941
:108FFE00E004F080C4E49002A9F09002A9E0C394CA
:10900E0008505AE4A3F09002AAE0C394085046A276
:10901E009092789002A9E0FF24F3F582E43407F5EC
:10902E0083E0FEC313FE3078047D8080027D00EE67
:10903E004DFE74F32FF582E43407F583EEF0900EB7
:10904E001AE0FF441890F800F0EF54F7F09002AADF
:10905E00E004F080B19002A9E004F0809D900E1A19
:0B906E00E054E7F090F800F0D2AF22D1
:1090790020060302913FE49002ADF09002ADE0FFBB
:10908900C39410501474542FF582E4340AF583E420
:10909900F09002ADE004F080E2E49002ADF09002BD
:1090A900ADE0FFC394025061EF2434FFE43446FE7F
:1090B9007D017C007B107A0012096E9002ADE024DC
:1090C9002FFFE43446FE12096E9002ADE0242CFF16
:1090D900E43446FE12096E9002ADE02423FFE43425
:1090E90046FE12096E9002ADE02426FFE43446FEE6
:1090F90012096E9002ADE02429FFE43446FE1209FC
:109109006E9002ADE004F08095E49002ADF090021B
:10911900ADE0FFC3940940030292BDEF2437FFE499
:109129003446FE7D017C007B107A0012096E9002A4
:10913900ADE004F080D8E49002ADF09002ADE0FF1C
:10914900C39410501574542FF582E4340AF58374CE
:10915900FFF09002ADE004F080E19007FCE0B40775
:109169000040030292BD909176F828287302918BF2
:109179000291B80291E502921202923F02926902AB
:109189009293E49002ADF09002ADE0FFC3940240E7
:10919900030292BDEF2429FFE43446FE7D017C00E1
:1091A9007B107A0012096E9002ADE004F080D8E4D9
:1091B9009002ADF09002ADE0FFC394024003029229
:1091C900BDEF2426FFE43446FE7D017C007B107A46
:1091D9000012096E9002ADE004F080D8E49002AD6F
:1091E900F09002ADE0FFC3940240030292BDEF2468
:1091F90023FFE43446FE7D017C007B107A001209CE
:109209006E9002ADE004F080D8E49002ADF09002D7
:10921900ADE0FFC3940240030292BDEF242CFFE4AA
:109229003446FE7D017C007B107A0012096E9002A3
:10923900ADE004F080D8E49002ADF09002ADE0FF1B
:10924900C39402506FEF242FFFE43446FE7D017C66
:10925900007B107A0012096E9002ADE004F080DB09
:10926900E49002ADF09002ADE0FFC394095045EFE0
:109279002437FFE43446FE7D017C007B107A00121E
:10928900096E9002ADE004F080DBE49002ADF0904D
:1092990002ADE0FFC39402501BEF2434FFE43446CF
:1092A900FE7D017C007B107A0012096E9002ADE010
:0592B90004F080DB223F
:1092BE00E49002B5F09002B5E0C39407502EE0FFA3
:1092CE0024F3F582E43407F583E0FEC4540F75F001
:1092DE000AA4FDEE540F2DFE74AE2FF582E4340277
:1092EE00F583EEF09002B5E004F080C99007FCE043
:1092FE00B4070040030293B790930DF82828730229
:10930E00932202933902934E02936302937902934E
:10931E008F0293A49002AEE0C3943B5006E004F09B
:10932E000293B7E49002AEF00293B79002AFE0C39F
:10933E00943B5005E004F08070E49002AFF0806939
:10934E009002B0E0C394175005E004F0805BE49007
:10935E0002B0F080549002B1E0C3941F5005E004B7
:10936E00F080469002B17401F0803E9002B2E0C3EC
:10937E00940C5005E004F080309002B27401F0803D
:10938E00289002B3E0C394065005E004F0801AE47E
:10939E009002B3F080139002B4E0C394635005E0E2
:1093AE0004F08005E49002B4F0E49002B5F090026F
:1093BE00B5E0C394075033E0FF24AEF582E43402E7
:1093CE00F583E0FE75F00A84FDC454F0FDEE75F0F1
:1093DE000A84E5F02DFE74F32FF582E43407F5834D
:0B93EE00EEF09002B5E004F080C42215
:1093F900E49002BDF09002BDE0C39407502EE0FF57
:1094090024F3F582E43407F583E0FEC4540F75F0C4
:109419000AA4FDEE540F2DFE74B62FF582E4340232
:10942900F583EEF09002BDE004F080C99007FCE0FE
:10943900B407004003029507909448F8282873025E
:10944900945D02947502948D0294A30294B90294D6
:10945900CF0294F39002B6E0D394014006E014F0F1
:109469000295079002B6743BF00295079002B7E0A7
:10947900D394014006E014F00295079002B7743BBB
:10948900F00295079002B8E0D394014005E014F08A
:10949900806C9002B87417F080649002B9E0D3949C
:1094A900014005E014F080569002B9741FF0804E17
:1094B9009002BAE0D394014005E014F08040900294
:1094C900BA740CF080389002BBE0FFD394064004D4
:1094D900E4F0802AEFD3940040089002BBE014F036
:1094E900801C9002BB7406F080149002BCE0D394F7
:1094F900004005E014F080069002BC7463F0E4902B
:1095090002BDF09002BDE0C394075033E0FF24B6DA
:10951900F582E43402F583E0FE75F00A84FDC45453
:10952900F0FDEE75F00A84E5F02DFE74F32FF58257
:10953900E43407F583EEF09002BDE004F080C42224
:10954900E49002C0F0A3F07F011266201238039064
:1095590002D3E4F0A37452F0A3E4F0A37475F0A36A
:10956900E4F0A3746EF0A3E4F0A37420F0A3E4F094
:10957900A37453F0A3E4F0A37465F0A3E4F0A37417
:109589006CF0A3E4F0A37466F0A3E4F0A37474F0A0
:10959900A3E4F0A37465F0A3E4F0A37473F0A3E467
:1095A900F0A37474F0A3E4F0A37431F0A3E4F0A37E
:1095B900742EF0A3E4F0A3742EF0A3E4F0A3742EA8
:1095C900F0A3E4F0A3742EF0E4A3F0A3F07FF87EF7
:1095D900031210D87B027AF279008B3E8A3F8940C8
:1095E900E92401F9E43A8B3EF53F89409002C0E055
:1095F900FEA3E0FF64274E601AEF64364E6014AB99
:109609003EAA3FA94012BBB1FF9002C0E4F0A3EF0C
:10961900F080D97F141201DD9002D3E4F0A37446DF
:10962900F0A3E4F0A37469F0A3E4F0A3746EF0A3CB
:10963900E4F0A37469F0A3E4F0A37473F0A3E4F075
:10964900A37468F0A3E4F0A37421F0E4A3F0A3F0F9
:109659007F097E041210D8753E02753FF2754000ED
:10966900754102754208754303E49002BEF0A3F008
:10967900C39002BEE094025034AB3E0540E540AAD7
:109689003F7002053F14F912BBB1FFAB410543E539
:1096990043AA427002054214F9EF12BBCC9002BFF3
:1096A900E004F070069002BEE004F080C39009E87F
:1096B900E024FC70030297481470030297EC24021B
:1096C90060030298849002D3E4F0A3743EF0A3E40B
:1096D900F0A3743EF0A3E4F0A37453F0A3E4F0A361
:1096E9007465F0A3E4F0A3746CF0A3E4F0A37466CA
:1096F900F0A3E4F0A37474F0A3E4F0A37465F0A3F9
:10970900E4F0A37473F0A3E4F0A37474F0A3E4F099
:10971900A37431F0A3E4F0A37420F0A3E4F0A374DC
:109729004FF0A3E4F0A3744BF0A3E4F0A37421F089
:10973900E4A3F0A3F07F187E071210D802991E90B7
:1097490002D3E4F0A3743EF0A3E4F0A3743EF0A3C3
:10975900E4F0A37444F0A3E4F0A37465F0A3E4F087
:10976900A37474F0A3E4F0A37465F0A3E4F0A37404
:1097790063F0A3E4F0A37474F0A3E4F0A37465F0B8
:10978900A3E4F0A37464F0A3E4F0A37420F0A3E4C9
:10979900F0A37431F0A3E4F0A37420F0A3E4F0A3E0
:1097A9007477F0A3E4F0A37461F0A3E4F0A37472F6
:1097B900F0A3E4F0A3746EF0A3E4F0A37469F0A33A
:1097C900E4F0A3746EF0A3E4F0A37467F0A3E4F0EB
:1097D900A37421F0E4A3F0A3F07F187E071210D838
:1097E90002991E9002D3E4F0A3743EF0A3E4F0A31F
:1097F900743EF0A3E4F0A37453F0A3E4F0A37465FA
:10980900F0A3E4F0A3746CF0A3E4F0A37466F0A3EE
:10981900E4F0A37474F0A3E4F0A37465F0A3E4F096
:10982900A37473F0A3E4F0A37474F0A3E4F0A37435
:1098390031F0A3E4F0A37420F0A3E4F0A37466F07C
:10984900A3E4F0A37461F0A3E4F0A37469F0A3E4C2
:10985900F0A3746CF0A3E4F0A37475F0A3E4F0A38F
:109869007472F0A3E4F0A37465F0A3E4F0A3742187
:10987900F07F187E071210D802991E9002D3E4F0E7
:10988900A3743EF0A3E4F0A3743EF0A3E4F0A37440
:1098990053F0A3E4F0A37465F0A3E4F0A3746CF0AF
:1098A900A3E4F0A37466F0A3E4F0A37474F0A3E452
:1098B900F0A37465F0A3E4F0A37473F0A3E4F0A338
:1098C9007474F0A3E4F0A37431F0A3E4F0A374205A
:1098D900F0A3E4F0A37466F0A3E4F0A37461F0A329
:1098E900E4F0A37469F0A3E4F0A3746CF0A3E4F0CA
:1098F900A37475F0A3E4F0A37472F0A3E4F0A37465
:1099090065F0A3E4F0A37421F0E4A3F0A3F07F18B9
:109919007E071210D87F0A1201DD1265B27F02128A
:0699290066209002D3E469
:10992F00F0A37452F0A3E4F0A37475F0A3E4F0A3D2
:10993F00746EF0A3E4F0A37420F0A3E4F0A37453C7
:10994F00F0A3E4F0A37465F0A3E4F0A3746CF0A3A8
:10995F00E4F0A37466F0A3E4F0A37474F0A3E4F04E
:10996F00A37465F0A3E4F0A37473F0A3E4F0A374FD
:10997F0074F0A3E4F0A37432F0A3E4F0A3742EF018
:10998F00A3E4F0A3742EF0A3E4F0A3742EF0A3E4E9
:10999F00F0A3742EF0E4A3F0A3F07F387E0A121028
:1099AF00D87B027AF279008B3E8A3F8940E9240105
:1099BF00F9E43A8B3EF53F89409002C0E0FEA3E008
:1099CF00FF64274E601AEF64364E6014AB3EAA3F19
:1099DF00A94012BBB1FF9002C0E4F0A3EFF080D911
:1099EF007F1E1201DD9002D3E4F0A37446F0A3E4CE
:1099FF00F0A37469F0A3E4F0A3746EF0A3E4F0A3F2
:109A0F007469F0A3E4F0A37473F0A3E4F0A3746893
:109A1F00F0A3E4F0A37421F0E4A3F0A3F07F497E58
:109A2F000A1210D8753E02753FF27540007541025B
:109A3F00754208754303E49002BEF0A3F0C3900291
:109A4F00BEE094025034AB3E0540E540AA3F7002A1
:109A5F00053F14F912BBB1FFAB410543E543AA42E1
:109A6F007002054214F9EF12BBCC9002BFE004F074
:109A7F0070069002BEE004F080C39009E8E064270E
:109A8F0070799002D3F0A3743EF0A3E4F0A3743E78
:109A9F00F0A3E4F0A37453F0A3E4F0A37465F0A370
:109AAF00E4F0A3746CF0A3E4F0A37466F0A3E4F005
:109ABF00A37474F0A3E4F0A37465F0A3E4F0A374AB
:109ACF0073F0A3E4F0A37474F0A3E4F0A37432F082
:109ADF00A3E4F0A37420F0A3E4F0A3744FF0A3E485
:109AEF00F0A3744BF0A3E4F0A37421F0E4A3F0A36C
:109AFF00F07F587E0D1210D8029BA49002D3E4F091
:109B0F00A3743EF0A3E4F0A3743EF0A3E4F0A374B7
:109B1F0053F0A3E4F0A37465F0A3E4F0A3746CF026
:109B2F00A3E4F0A37466F0A3E4F0A37474F0A3E4C9
:109B3F00F0A37465F0A3E4F0A37473F0A3E4F0A3AF
:109B4F007474F0A3E4F0A37432F0A3E4F0A37420D0
:109B5F00F0A3E4F0A37466F0A3E4F0A37461F0A3A0
:109B6F00E4F0A37469F0A3E4F0A3746CF0A3E4F041
:109B7F00A37475F0A3E4F0A37472F0A3E4F0A374DC
:109B8F0065F0A3E4F0A37421F0E4A3F0A3F07F58F1
:109B9F007E0D1210D87F0A1201DD1265B27F0312FB
:109BAF0066209002D3E4F0A37452F0A3E4F0A37400
:109BBF0075F0A3E4F0A3746EF0A3E4F0A37420F0A7
:109BCF00A3E4F0A37453F0A3E4F0A37465F0A3E44B
:109BDF00F0A3746CF0A3E4F0A37466F0A3E4F0A315
:109BEF007474F0A3E4F0A37465F0A3E4F0A37473AA
:109BFF00F0A3E4F0A37474F0A3E4F0A37433F0A320
:109C0F00E4F0A3742EF0A3E4F0A3742EF0A3E4F019
:109C1F00A3742EF0A3E4F0A3742EF0E4A3F0A3F04A
:109C2F007F787E101210D87B027AF279008B3E8AF1
:109C3F003F8940E92401F9E43A8B3EF53F89409092
:109C4F0002C0E0FEA3E0FF64274E601AEF64364EB9
:109C5F006014AB3EAA3FA94012BBB1FF9002C0E413
:109C6F00F0A3EFF080D97F141201DD9002D3E4F05E
:109C7F00A37446F0A3E4F0A37469F0A3E4F0A37413
:109C8F006EF0A3E4F0A37469F0A3E4F0A37473F08F
:109C9F00A3E4F0A37468F0A3E4F0A37421F0E4A3A9
:109CAF00F0A3F07F897E101210D8753E02753FF237
:109CBF00754000754102754208754303E49002BE7A
:109CCF00F0A3F0C39002BEE094025034AB3E0540C7
:109CDF00E540AA3F7002053F14F912BBB1FFAB413B
:109CEF000543E543AA427002054214F9EF12BBCCBB
:109CFF009002BFE004F070069002BEE004F080C353
:069D0F009009E8E0642762
:109D150070779002D3F0A3743EF0A3E4F0A3743EF1
:109D2500F0A3E4F0A37453F0A3E4F0A37465F0A3E7
:109D3500E4F0A3746CF0A3E4F0A37466F0A3E4F07C
:109D4500A37474F0A3E4F0A37465F0A3E4F0A37422
:109D550073F0A3E4F0A37474F0A3E4F0A37433F0F8
:109D6500A3E4F0A37420F0A3E4F0A3744FF0A3E4FC
:109D7500F0A3744BF0A3E4F0A37421F0E4A3F0A3E3
:109D8500F07F987E131210D8229002D3E4F0A374CA
:109D95003EF0A3E4F0A3743EF0A3E4F0A37453F003
:109DA500A3E4F0A37465F0A3E4F0A3746CF0A3E45A
:109DB500F0A37466F0A3E4F0A37474F0A3E4F0A335
:109DC5007465F0A3E4F0A37473F0A3E4F0A37474D2
:109DD500F0A3E4F0A37433F0A3E4F0A37420F0A39C
:109DE500E4F0A37466F0A3E4F0A37461F0A3E4F0D7
:109DF500A37469F0A3E4F0A3746CF0A3E4F0A37476
:109E050075F0A3E4F0A37472F0A3E4F0A37465F015
:109E1500A3E4F0A37421F0E4A3F0A3F07F987E13EC
:049E25001210D8221D
:109E2900E49002C2F0900A2DE0FF9002C2E0FEC366
:109E39009F501D75F002EEA424D3F582E5F034029B
:109E4900F583E4F0A37412F09002C2E004F080D527
:109E59009002C2E0FFC3940C501D75F002EFA424D8
:109E6900D3F582E5F03402F583E4F0A37420F09091
:109E790002C2E004F080D9E49002EBF0A3F07F1273
:109E8900FE1210D8200A10900A2DE0C3940C500439
:109E9900E004F022D20A22900A2DE0D39400400473
:079EA900E014F022C20A22BE
:109EB0007B027A1679098B338A34893512BBB190CB
:109EC00007DBF0F46002E4F07B027A16790A8B3348
:109ED0008A34893512BBB19002CCF0098B338A34B5
:109EE000893512BBB1FE3395E0900A17F0A3CEF08E
:109EF000120274900A5274FAF01266A69002D3E429
:109F0000F0A37416F0A3E4F0A37417F0A3E4F0A395
:109F1000741AF0A3E4F0A37419F0E4A3F0A3F07FA3
:109F20006C7E091213229002D3E4F0A3741BF0A3F9
:109F3000E4F0A37418F0A3E4F0A3741AF0A3E4F01F
:109F4000A3741BF0A3E4F0A3741CF0A3E4F0A374C7
:109F50001AF0A3E4F0A37418F0A3E4F0A3741BF0C8
:109F6000E4A3F0A3F07F167E0E1213229002D3E436
:109F7000F0A3744DF0A3E4F0A3746FF0A3E4F0A396
:109F80007464F0A3E4F0A37465F0A3E4F0A3746C2C
:109F9000F0A3E4F0A3743AF0A3E4F0A37420F0A3D8
:109FA000E4F0A37450F0A3E4F0A37461F0A3E4F030
:109FB000A37472F0A3E4F0A37461F0A3E4F0A374BB
:109FC00053F0A3E4F0A37463F0A3E4F0A3746FF080
:109FD000A3E4F0A37470F0A3E4F0A37465F0E4A329
:109FE000F0A3F07FCC7E121210D89002D3E4F0A33D
:109FF0007456F0A3E4F0A37465F0A3E4F0A37472C4
:10A00000F0A3E4F0A37473F0A3E4F0A37469F0A3E5
:10A01000E4F0A3746FF0A3E4F0A3746EF0A3E4F093
:10A02000A3743AF0A3E4F0A37420F0A3E4F0A374C3
:10A0300032F0A3E4F0A3742EF0A3E4F0A37430F0A4
:10A04000A3E4F0A37436F0E4A3F0A3F07FEC7E1554
:10A050001210D89002D3E4F0A37446F0A3E4F0A366
:10A060007472F0A3E4F0A37465F0A3E4F0A3746445
:10A07000F0A3E4F0A37465F0A3E4F0A37472F0A37A
:10A08000E4F0A37469F0A3E4F0A37463F0A3E4F034
:10A09000A3746BF0A3E4F0A37420F0A3E4F0A37422
:10A0A00045F0A3E4F0A3746EF0A3E4F0A37467F0AA
:10A0B000A3E4F0A37469F0A3E4F0A3746EF0A3E446
:10A0C000F0A37465F0A3E4F0A37465F0A3E4F0A337
:10A0D0007472F0A3E4F0A37469F0A3E4F0A3746EC7
:10A0E000F0A3E4F0A37467F0A3E4F0A37420F0A35A
:10A0F000E4F0A37449F0A3E4F0A3746EF0A3E4F0D9
:10A10000A37463F0A3E4F0A3742EF0A3E4F0A374AB
:10A1100020F0A3E4F0A37455F0A3E4F0A37453F08B
:10A12000A3E4F0A37441F0E4A3F0A3F07F037E194D
:10A130001210D89002D3E4F0A37441F0A3E4F0A38A
:10A140007470F0A3E4F0A37472F0A3E4F0A3746954
:10A15000F0A3E4F0A3746CF0A3E4F0A37420F0A3E4
:10A16000E4F0A37432F0A3E4F0A37430F0A3E4F0BD
:10A17000A37430F0A3E4F0A37433F0E4A3F0A3F0ED
:10A180007F2D7E1C1210D87F1E1201DD7B027A16F5
:10A1900079088B338A34893512BBB1900A52F0D3D7
:10A1A0006480948A5008E0C364809476500EE490F2
:10A1B0000A52F0AB33AA34A93512BBCC1266A622E0
:10A1C000900E1AE0543F4480F0900E20E0FF6013A0
:10A1D000900E1AE04440F09002CEE0C394FA50038F
:10A1E000E004F09007D3E060229002CEE0D3941E0A
:10A1F0005003EF7011900E1AE0547FF01201997F16
:10A20000021201DD80057F051201DD900E1AE0903B
:04A21000F800F02240
:10A21400900A27E054F84401F090F1FCF0E4900235
:10A22400C3F09002C3E0C39464502E900A27E05414
:10A23400FEF090F1FCF09002C47405F09002C4E0CA
:10A24400FF14F0EF70F6900A27E04401F090F1FC5F
:10A25400F09002C3E004F080C9900A27E054F84467
:10A2640003F090F1FCF09002C4740AF09002C4E090
:10A27400FF14F0EF70F6E49002C3F020B34C9002A8
:10A28400C3E0C39446504320B3409002C4740AF020
:10A294009002C4E0FF14F0EF70F620B32D900A276B
:10A2A400E054FEF090F1FCF04401900A27F090F1A4
:10A2B400FCF09002C4740AF09002C4E0FF14F0EFC2
:10A2C40070F69002C3E004F080B1900A27E054F8DD
:10A2D4004401F090F1FCF0E49002C5F09002C5E076
:10A2E400C39464501D900A27E054FEF090F1FCF0F2
:10A2F4004401900A27F090F1FCF09002C5E004F0CC
:10A3040080DA900E1DE06009900A27E0440FF08087
:10A3140009900A27E054F74407F0900A27E090F1E7
:10A32400FCF0900A28E0FF9002C3E0FE6F70030285
:10A33400A43F900A28EEF0E49002C5F09002C5E034
:10A34400FFC3940D501474542FF582E4340AF5833A
:10A35400E4F09002C5E004F080E2E49002C6F090DC
:10A3640002C6E0FFC39405501BEF2417FFE43443F7
:10A37400FE7D017C007B0D7A0012096E9002C6E01E
:10A3840004F080DB9002C3E0FFD394365006A3743C
:10A3940006F0804BEFD3943850089002C47405F053
:10A3A400803DEFD3943A50089002C47404F0802F97
:10A3B400EFD3943C50089002C47403F08021EFD38F
:10A3C400943E50089002C47402F08013EFD394407A
:10A3D40050089002C47401F08005E49002C4F09027
:10A3E40002C4E0D3940540037405F0E49002C3F082
:10A3F4009002C3E0FFC3940D501574542FF582E40A
:10A40400340AF583747EF09002C3E004F080E1E442
:10A414009002C5F09002C4E0FFA3E0FEC39F501B6E
:10A42400EE2417FFE43443FE7D017C007B0D7A00AB
:0CA4340012096E9002C5E004F080D922ED
:10A4400075420275430A754454E49002C7F09002C5
:10A45000C7E0FFC39405501574542FF582E4340A05
:10A46000F58374FFF09002C7E004F080E17FC77EBF
:10A47000427D037C007B057A0012096E7F477E4592
:10A4800012096EE49002C7F09002C7E0FFC3941176
:10A49000501574542FF582E4340AF5837401F0905A
:10A4A00002C7E004F080E17FC67E427D017C007B34
:10A4B000117A0012096E75420275430A754454E41C
:10A4C0009002C7F09002C7E0C39405501BAB420551
:10A4D00044E544AA437002054314F9748012BBCCCE
:10A4E0009002C7E004F080DCAB420544E544AA4397
:10A4F0007002054314F974F812BBCCE49002C7F063
:10A500009002C7E0C39405501BAB420544E544AA42
:10A51000437002054314F9748812BBCC9002C7E063
:10A5200004F080DCAB420544E544AA4370020543D5
:10A5300014F974F812BBCCE49002C7F09002C7E0A3
:10A54000C39405501BAB420544E544AA4370020581
:10A550004314F9748012BBCC9002C7E004F080DC95
:10A560007FCC7E427D017C007B117A0012096E2235
:10A681000000386CC6C6C6C6C6C6C6C66C38000051
:10A69100000008381818181818181818183C000065
:10A6A1000000386CC6C606060C08103262FE0000B7
:10A6B1000000386CC6060C180C0606C66C38000083
:10A6C10000040C1C3C2C6CCCCC8CFE0C0C1E000031
:10A6D1000000FEC0C0C0F8EC060606C66C380000DB
:10A6E1000000386CC6C0D8ECC6C6C6C66C380000BF
:10A6F1000000FEFE82060C0C1818303030300000CD
:10A701000000386CC6C66C386CC6C6C66C38000012
:10A711000000386CC6C6C6C66E3E06C66C38000060
:10A72100000007081020202020202010080700002A
:10A731000000E010080404040404040810E0000010
:10A741000000070F1F3F3F3F3F3F3F1F0F07000024
:10A751000000E0F0F8FCFCFCFCFCFCF8F0E0000080
:10A761000000FEC2C0C0C4FCC4C0C0C0C2FE000024
:10A771000000FEC2C0C0C4FCC4C0C0C0C0E0000034
:10A781000000000002060E1E0E060200000000007E
:10A7910000000000080C0E0F0E0C08000000000065
:10A7A100000000007E7E7E7E7E7E7E7E00000000B8
:10A7B10008080808080808FF080808080808080821
:10A7C10000003F202020202028342221203F0000AB
:10A7D1000000FC0404040C142444840404FC000060
:10A7E100000000030404041F1F1F1F1F1F0000009F
:10A7F100000000C0202020F8F8F8F8F8F800000068
:10A8010000003F202020202020202020203F000089
:10A811000000FC04040404040404040404FC000017
:10A82100000103070F1F3F7F070707070707000006
:10A83100000080C0E0F0F8FCC0C0C0C0C0C0000093
:10A8410000003F3F3F3F3F3F3F3F3F3F3F3F000013
:10A851000000FCFCFCFCFCFCFCFCFCFCFCFC000027
:10A861000000081C3E7F08080808080808080808B6
:10A87100FFFFFFFFFFFFFFFFFFFFFFFFFFFFFFFFE7
:10A8810000000000000000000000000000000000C7
:10A891000000183C3C3C1818180018180000000073
:10A8A1000066666624000000000000000000000051
:10A8B1000000006C6CFE6C6C6CFE6C6C00000000A7
:10A8C10018187CC6C2C07C060686C67C1818000013
:10A8D10000000000C2C60C183060C68600000000EF
:10A8E1000000386C6C3876DCCCCCCC7600000000F3
:10A8F1000030303060000000000000000000000067
:10A9010000000C18303030303030180C00000000DE
:10A91100000030180C0C0C0C0C0C1830000000005E
:10A921000000000000663CFF3C66000000000000E3
:10A93100000000000018187E181800000000000038
:10A94100000000000000000000181818300000008E
:10A9510000000000000000FE0000000000000000F8
:10A9610000000000000000000000181800000000B6
:10A971000000000002060C183060C08000000000DA
:10A981000000386CC6C6D6D6C6C66C3800000000BA
:10A9910000001838781818181818187E00000000E0
:10A9A10000007CC6060C183060C0C6FE0000000026
:10A9B10000007CC606063C060606C67C00000000B8
:10A9C10000000C1C3C6CCCFE0C0C0C1E00000000AA
:10A9D1000000FEC0C0C0FC060606C67C00000000E8
:10A9E10000003860C0C0FCC6C6C6C67C00000000BE
:10A9F1000000FEC606060C183030303000000000A2
:10AA010000007CC6C6C67CC6C6C6C67C0000000067
:10AA110000007CC6C6C67E0606060C780000000053
:10AA210000000000181800000018180000000000C5
:10AA31000000000018180000001818300000000085
:10AA4100000000060C18306030180C0600000000F1
:10AA510000000000007E00007E00000000000000F9
:06AA610000000060301847
:10AA67000C060C1830600000000000007CC6C60C05
:10AA7700181818001818000000000000007CC6C64F
:10AA8700DEDEDEDCC07C00000000000010386CC693
:10AA9700C6FEC6C6C6C6000000000000FC666666A5
:10AAA7007C66666666FC0000000000003C66C2C06B
:10AAB700C0C0C0C2663C000000000000F86C6666BB
:10AAC700666666666CF8000000000000FE66626855
:10AAD7007868606266FE000000000000FE6662683B
:10AAE7007868606060F00000000000003C66C2C04B
:10AAF700C0DEC6C6663A000000000000C6C6C6C66D
:10AB0700FEC6C6C6C6C60000000000003C181818DE
:10AB170018181818183C0000000000001E0C0C0C38
:10AB27000C0CCCCCCC78000000000000E666666C0C
:10AB370078786C6666E6000000000000F0606060F0
:10AB47006060606266FE000000000000C6EEFEFE68
:10AB5700D6C6C6C6C6C6000000000000C6E6F6FE9A
:10AB6700DECEC6C6C6C60000000000007CC6C6C64C
:10AB7700C6C6C6C6C67C000000000000FC66666646
:10AB87007C60606060F00000000000007CC6C6C604
:10AB9700C6C6C6D6DE7C0C0E00000000FC666666E4
:10ABA7007C6C666666E60000000000007CC6C66036
:10ABB700380C06C6C67C0000000000007E7E5A18CE
:10ABC70018181818183C000000000000C6C6C6C6B2
:10ABD700C6C6C6C6C67C000000000000C6C6C6C6FC
:10ABE700C6C6C66C3810000000000000C6C6C6C640
:10ABF700D6D6D6FEEE6C000000000000C6C66C7C00
:10AC070038387C6CC6C600000000000066666666C1
:10AC17003C181818183C000000000000FEC6860CFF
:10AC2700183060C2C6FE000000000000000070403F
:10AC3700404040404040700000000000000080405D
:10AC4700404020201010100000000000000070108D
:10AC570010101010101070000000000000002020DD
:10AC67005088000000000000000000000000000005
:10AC7700000000000000F8000000000000002010A5
:10AC87000000000000000000000000000000007845
:10AC97000C7CCCCCCC76000000000000E060607833
:10ACA7006C666666667C0000000000000000007CA1
:10ACB700C6C0C0C0C67C0000000000001C0C0C3CD5
:10ACC7006CCCCCCCCC760000000000000000007CEF
:10ACD700C6FEC0C0C67C000000000000386C64607F
:10ACE700F060606060F00000000000000000007687
:10ACF700CCCCCCCCCC7C0CCC78000000E060606C79
:10AD07007666666666E600000000000018180038E0
:10AD170018181818183C0000000000000606000E5E
:10AD270006060606060666663C000000E0606066EA
:10AD37006C78786C66E60000000000003818181878
:10AD470018181818183C000000000000000000EC5C
:10AD5700FED6D6D6D6C6000000000000000000DCF4
:10AD67006666666666660000000000000000007CFC
:10AD7700C6C6C6C6C67C000000000000000000DC96
:10AD870066666666667C6060F0000000000000761C
:10AD9700CCCCCCCCCC7C0C0C1E000000000000DC22
:10ADA7007666606060F00000000000000000007C34
:10ADB700C660380CC67C000000000000103030FC74
:10ADC70030303030361C000000000000000000CC9E
:10ADD700CCCCCCCCCC760000000000000000006694
:10ADE700666666663C18000000000000000000C6AA
:10ADF700C6D6D6D6FE6C000000000000000000C6D4
:10AE07006C3838386CC6000000000000000000C62F
:10AE1700C6C6C6C6C67E060CF8000000000000FEC7
:10AE2700CC183060C6FE0000000000000E1818188D
:10AE370070181818180E00000000000018181818CD
:06AE47000018181818188D
:10AE4D00000000000000701818180E18181818705F
:10AE5D0000000000000076DC000000000000000093
:10AE6D0000000000000000000000000000000007CE
:10AE7D0007000000000000000000000000000000BE
:10AE8D0000000000000000FFFF00000000000000B7
:10AE9D00000000000000000000000000000000E0C5
:10AEAD00E000000000000000000000000000000FA6
:10AEBD00070303037F330206040C18100100000082
:10AECD00001F0000000078F223233FFF232363605F
:10AEDD006038181FFFD81818FFE0000060303030C0
:10AEED003030303030303030F0602080800000F075
:10AEFD00F8180000000003030306060C083F3F038B
:10AF0D0002071F1800011F3C300000000C0E0C0C36
:10AF1D0004044567FE86830F3EC3010161C70C38EB
:10AF2D0000000000000060703000E0800070E080E4
:10AF3D003070E0C08082C2663E1E0E00000000012F
:10AF4D001F18080B0F030333331212131F3CF0406D
:10AF5D0000000000000303C7E6C7CC88183703C301
:10AF6D00060C18B07FB81018191F0800000000005B
:10AF7D00E0F0E0C0C0800080C0703EDFE070606037
:10AF8D00E0E00000000000000C0F05000031311161
:10AF9D00050D0919183030110304000000000000E0
:10AFAD003CEE8C8CBCACACACA4ACEC64705CCC86D4
:10AFBD000000000000101C1C181818D8D8D898D8FC
:10AFCD00D8D8D8080C0C0C7C3C1C080000000007DD
:10AFDD000301000000077F760606060607070E0E22
:10AFED000C0000000007030383830301031F3D01D1
:10AFFD00063E78189B1EF86000000000000000302F
:10B00D0038180060F0C080808080C0C04062323A45
:10B01D001E0E070000030303030706060C0E1E3663
:10B02D0026468606060606060606000000008098DF
:10B03D001C0C0400603019090D0703070F1C7080EC
:10B04D0000000000000000C0E0E0E0C0C0C0808053
:10B05D0080000080C0E07C3F1E000000000000006A
:10B06D0000000000000000000101010303060F1F96
:10B07D0000000000000000181C1C3C3E2E6FC7C7CE
:10B08D0083FFFF01000000830000000000000000AE
:10B09D0000000000000000808080C0E0E0E0F0F8DB
:10B0AD00000000000000000F03010101010101017A
:10B0BD00010101010101030F00000000000000FC6F
:10B0CD00FFC7C3C3C3C3FFFEC7C3C1C1C1C3FFFC19
:10B0DD0000000000000000000080808080800000E3
:10B0ED0080C0C0C0C0C08000000000000000000F84
:10B0FD000301010101010101010101010101070F1D
:10B10D0000000000000000FCFF87838180808080AC
:10B11D0080808081838FFFF8000000000000000018
:10B12D000080C0E0E0F0707070F0F0E0C0C0000092
:10B13D0000000000000000000001010101010000FD
:10B14D000000010101010101000000000000007D6F
:10B15D00E7C381C1C0F8FC7E1F0703018181FF3E5B
:10B16D0000000000000000000000000000000000D2
:10B17D000080C0C0C08080000000000000000007FB
:10B18D000301010101010101010101010101030798
:10B19D0000000000000000F0E0C0C0C0C0C0C0C092
:10B1AD00C0C0C0C0C0C0FFFF000000000000000014
:10B1BD0000000000000000000000002060C0C08002
:10B1CD00000000000000000000000000000000076B
:10B1DD00070000000000000000000000000000005B
:10B1ED0000000000000000FFFF0000000000000054
:10B1FD00000000000000000000000000000000E062
:10B20D00E000000000000000000000000000000051
:10B21D000000000000000000000000000000000021
:06B22D000000000000001B
:10B23300000C3C7C1C1C1C1C1C1C1C1C1C1C1C1CF7
:10B243001C7F000000000000000000000000000060
:10B2530000000000000000000000000000000000EB
:10B26300000000010307070F0F0F0F0F0707070366
:10B273000100000000000000007FE3808000000068
:10B283000000000000008080E37F00000000000059
:10B29300000080C0E0707078787878787070F0E0A3
:10B2A300C0000000000000000007070604000000C3
:10B2B300000000000000000000000000000000008B
:10B2C30000FFFF1C1C1C1C1C1C1C1C1C1C1C1C1C11
:10B2D3003E7F00000000000000F0F030100000008E
:10B2E300000000000000000000000000000000005B
:10B2F300000000000000000101030303030101013A
:10B30300000000000000000000071C3870E0C0DCF3
:10B31300FFC78383838383C3E77E000000000000AD
:10B32300000000000000000000808080808080809A
:10B333000000000000000000000000010100000008
:10B3430000000000000000000100000000000000F9
:10B353000078FEDE0E06060C1C7E0F070303070EA5
:10B36300FCF00000000000000000000000000000EE
:10B3730000000000000000000000000000000000CA
:10B3830000000001010101010101000000000000B3
:10B3930000030000000000000078CE8687878383C7
:10B3A30083C7FF77060E0C1870C000000000000072
:10B3B300000000000000000000000000000000008A
:10B3C3000000000000000000000000000001030373
:10B3D300060C18670000000103060C300000007023
:10B3E300180C86C6C3818000000FFFE363E3C383A9
:10B3F30007263E1E1C0000000000000000C0E0F80D
:10B403007F3F808000000000000000000000020376
:10B41300030101010101073F0307070F1B133363F7
:10B423008303030302000080808000010F4CCC0CD7
:10B433000F0ECCC848181830204000000000000050
:10B443000070F0C00000003FFEE0C0C0C0404040BC
:10B4530040606060404000000000000101030303FE
:10B4630003030303030301010000000000000000C5
:10B47300007CEEC78383838383838383838383C730
:10B48300EE7C0000000000000000000000808080CF
